Archive member included to satisfy reference by file (symbol)

d:/cc/arm-yagarto-5.4.2016q3/bin/../lib/gcc/arm-none-eabi/5.4.1/armv7-m\libgcc.a(_arm_addsubdf3.o)
                              obj/uc_libc_dev/stdio/stdio_uc.o (__aeabi_dsub)
d:/cc/arm-yagarto-5.4.2016q3/bin/../lib/gcc/arm-none-eabi/5.4.1/armv7-m\libgcc.a(_arm_muldivdf3.o)
                              obj/uc_libc_dev/_arch/arm_lpc/uart/uart0_irq.o (__aeabi_dmul)
d:/cc/arm-yagarto-5.4.2016q3/bin/../lib/gcc/arm-none-eabi/5.4.1/armv7-m\libgcc.a(_arm_cmpdf2.o)
                              obj/uc_libc_dev/stdio/stdio_uc.o (__aeabi_dcmpeq)
d:/cc/arm-yagarto-5.4.2016q3/bin/../lib/gcc/arm-none-eabi/5.4.1/armv7-m\libgcc.a(_arm_fixdfsi.o)
                              obj/uc_libc_dev/_arch/arm_lpc/uart/uart0_irq.o (__aeabi_d2iz)
d:/cc/arm-yagarto-5.4.2016q3/bin/../lib/gcc/arm-none-eabi/5.4.1/armv7-m\libgcc.a(_arm_addsubsf3.o)
                              obj/uc_libc_dev/_arch/arm_lpc/uart/uart0_irq.o (__aeabi_fadd)
d:/cc/arm-yagarto-5.4.2016q3/bin/../lib/gcc/arm-none-eabi/5.4.1/armv7-m\libgcc.a(_arm_muldivsf3.o)
                              obj/uc_libc_dev/_arch/arm_lpc/uart/uart0_irq.o (__aeabi_fmul)
d:/cc/arm-yagarto-5.4.2016q3/bin/../lib/gcc/arm-none-eabi/5.4.1/../../../../arm-none-eabi/lib/armv7-m\libc.a(lib_a-locale.o)
                              obj/uc_libc_dev/misc/utils.o (__locale_ctype_ptr)
d:/cc/arm-yagarto-5.4.2016q3/bin/../lib/gcc/arm-none-eabi/5.4.1/../../../../arm-none-eabi/lib/armv7-m\libc.a(lib_a-mbtowc_r.o)
                              d:/cc/arm-yagarto-5.4.2016q3/bin/../lib/gcc/arm-none-eabi/5.4.1/../../../../arm-none-eabi/lib/armv7-m\libc.a(lib_a-locale.o) (__ascii_mbtowc)
d:/cc/arm-yagarto-5.4.2016q3/bin/../lib/gcc/arm-none-eabi/5.4.1/../../../../arm-none-eabi/lib/armv7-m\libc.a(lib_a-memset.o)
                              obj/uc_libc_dev/cli/cli.o (memset)
d:/cc/arm-yagarto-5.4.2016q3/bin/../lib/gcc/arm-none-eabi/5.4.1/../../../../arm-none-eabi/lib/armv7-m\libc.a(lib_a-strcmp.o)
                              obj/prompt.o (strcmp)
d:/cc/arm-yagarto-5.4.2016q3/bin/../lib/gcc/arm-none-eabi/5.4.1/../../../../arm-none-eabi/lib/armv7-m\libc.a(lib_a-strlen-stub.o)
                              obj/uc_libc_dev/cli/cli.o (strlen)
d:/cc/arm-yagarto-5.4.2016q3/bin/../lib/gcc/arm-none-eabi/5.4.1/../../../../arm-none-eabi/lib/armv7-m\libc.a(lib_a-wctomb_r.o)
                              d:/cc/arm-yagarto-5.4.2016q3/bin/../lib/gcc/arm-none-eabi/5.4.1/../../../../arm-none-eabi/lib/armv7-m\libc.a(lib_a-locale.o) (__ascii_wctomb)
d:/cc/arm-yagarto-5.4.2016q3/bin/../lib/gcc/arm-none-eabi/5.4.1/../../../../arm-none-eabi/lib/armv7-m\libc.a(lib_a-ctype_.o)
                              d:/cc/arm-yagarto-5.4.2016q3/bin/../lib/gcc/arm-none-eabi/5.4.1/../../../../arm-none-eabi/lib/armv7-m\libc.a(lib_a-locale.o) (_ctype_)
d:/cc/arm-yagarto-5.4.2016q3/bin/../lib/gcc/arm-none-eabi/5.4.1/../../../../arm-none-eabi/lib/armv7-m\libc.a(lib_a-impure.o)
                              d:/cc/arm-yagarto-5.4.2016q3/bin/../lib/gcc/arm-none-eabi/5.4.1/../../../../arm-none-eabi/lib/armv7-m\libc.a(lib_a-locale.o) (_impure_ptr)

Allocating common symbols
Common symbol       size              file

_row_offsets        0x4               obj/uc_libc_dev/display/liquid_crystal.o
control             0x18              obj/main.o
_displaycontrol     0x1               obj/uc_libc_dev/display/liquid_crystal.o
_numlines           0x1               obj/uc_libc_dev/display/liquid_crystal.o
gkey_FastInc        0x4               obj/uc_libc_dev/keyboard/gkey.o
_displaymode        0x1               obj/uc_libc_dev/display/liquid_crystal.o
_displayfunction    0x1               obj/uc_libc_dev/display/liquid_crystal.o
_cols               0x1               obj/uc_libc_dev/display/liquid_crystal.o

Discarded input sections

 .text          0x00000000        0x0 obj/uc_libc_dev/_arch/arm_lpc/common/arm.o
 .data          0x00000000        0x0 obj/uc_libc_dev/_arch/arm_lpc/common/arm.o
 .bss           0x00000000        0x0 obj/uc_libc_dev/_arch/arm_lpc/common/arm.o
 .text._exit    0x00000000        0x2 obj/uc_libc_dev/_arch/arm_lpc/common/arm.o
 .text          0x00000000        0x0 obj/uc_libc_dev/_arch/arm_lpc/common/startup/startup.o
 .data          0x00000000        0x0 obj/uc_libc_dev/_arch/arm_lpc/common/startup/startup.o
 .bss           0x00000000        0x0 obj/uc_libc_dev/_arch/arm_lpc/common/startup/startup.o
 .text          0x00000000        0x0 obj/uc_libc_dev/_arch/arm_lpc/common/vic_cortexm3.o
 .data          0x00000000        0x0 obj/uc_libc_dev/_arch/arm_lpc/common/vic_cortexm3.o
 .bss           0x00000000        0x0 obj/uc_libc_dev/_arch/arm_lpc/common/vic_cortexm3.o
 .text.sysTick_ISR
                0x00000000       0x20 obj/uc_libc_dev/_arch/arm_lpc/common/vic_cortexm3.o
 .text.uart0_ISR
                0x00000000       0x20 obj/uc_libc_dev/_arch/arm_lpc/common/vic_cortexm3.o
 .text.nvic_disableIRQ
                0x00000000       0x18 obj/uc_libc_dev/_arch/arm_lpc/common/vic_cortexm3.o
 .text.nvic_getPendingIRQ
                0x00000000       0x22 obj/uc_libc_dev/_arch/arm_lpc/common/vic_cortexm3.o
 .text.nvic_getActiveIRQ
                0x00000000       0x22 obj/uc_libc_dev/_arch/arm_lpc/common/vic_cortexm3.o
 .text          0x00000000        0x0 obj/uc_libc_dev/_arch/arm_lpc/timer/systick.o
 .data          0x00000000        0x0 obj/uc_libc_dev/_arch/arm_lpc/timer/systick.o
 .bss           0x00000000        0x0 obj/uc_libc_dev/_arch/arm_lpc/timer/systick.o
 .text.systime_ClearIntHandler
                0x00000000        0xc obj/uc_libc_dev/_arch/arm_lpc/timer/systick.o
 .text.systime_GetTick
                0x00000000        0xc obj/uc_libc_dev/_arch/arm_lpc/timer/systick.o
 .text.systime_GetElapsedTick
                0x00000000        0xc obj/uc_libc_dev/_arch/arm_lpc/timer/systick.o
 .text.systime_Pause
                0x00000000       0x14 obj/uc_libc_dev/_arch/arm_lpc/timer/systick.o
 .text.timeout_Init
                0x00000000       0x1c obj/uc_libc_dev/_arch/arm_lpc/timer/systick.o
 .text.timeout_Check
                0x00000000       0x24 obj/uc_libc_dev/_arch/arm_lpc/timer/systick.o
 .bss.timerout  0x00000000        0x4 obj/uc_libc_dev/_arch/arm_lpc/timer/systick.o
 .bss.timerout_startTime
                0x00000000        0x4 obj/uc_libc_dev/_arch/arm_lpc/timer/systick.o
 .text          0x00000000        0x0 obj/uc_libc_dev/_arch/arm_lpc/timer/delay.o
 .data          0x00000000        0x0 obj/uc_libc_dev/_arch/arm_lpc/timer/delay.o
 .bss           0x00000000        0x0 obj/uc_libc_dev/_arch/arm_lpc/timer/delay.o
 .text          0x00000000        0x0 obj/uc_libc_dev/_arch/arm_lpc/uart/uart0_irq.o
 .data          0x00000000        0x0 obj/uc_libc_dev/_arch/arm_lpc/uart/uart0_irq.o
 .bss           0x00000000        0x0 obj/uc_libc_dev/_arch/arm_lpc/uart/uart0_irq.o
 .text.uart0_ClearBufferRx
                0x00000000       0x3c obj/uc_libc_dev/_arch/arm_lpc/uart/uart0_irq.o
 .text.uart0_CountRxOverflow
                0x00000000       0x10 obj/uc_libc_dev/_arch/arm_lpc/uart/uart0_irq.o
 .text.uart0_BufferRxIsEmpty
                0x00000000       0x14 obj/uc_libc_dev/_arch/arm_lpc/uart/uart0_irq.o
 .text.uart0_BufferQtdRx
                0x00000000        0xc obj/uc_libc_dev/_arch/arm_lpc/uart/uart0_irq.o
 .text.uart0_GetBufferRx
                0x00000000        0x8 obj/uc_libc_dev/_arch/arm_lpc/uart/uart0_irq.o
 .text.uart0_SpaceTx
                0x00000000       0x28 obj/uc_libc_dev/_arch/arm_lpc/uart/uart0_irq.o
 .text.uart0_FlushTx
                0x00000000       0x24 obj/uc_libc_dev/_arch/arm_lpc/uart/uart0_irq.o
 .text.uart0_EmptyTx
                0x00000000       0x18 obj/uc_libc_dev/_arch/arm_lpc/uart/uart0_irq.o
 .text.uart0_WriteTx
                0x00000000       0x2c obj/uc_libc_dev/_arch/arm_lpc/uart/uart0_irq.o
 .text.uart0_PutString
                0x00000000       0x18 obj/uc_libc_dev/_arch/arm_lpc/uart/uart0_irq.o
 .text          0x00000000        0x0 obj/main.o
 .data          0x00000000        0x0 obj/main.o
 .bss           0x00000000        0x0 obj/main.o
 .text          0x00000000        0x0 obj/app.o
 .data          0x00000000        0x0 obj/app.o
 .bss           0x00000000        0x0 obj/app.o
 .text          0x00000000        0x0 obj/prompt.o
 .data          0x00000000        0x0 obj/prompt.o
 .bss           0x00000000        0x0 obj/prompt.o
 .text          0x00000000        0x0 obj/uc_libc_dev/stdio/stdio_uc.o
 .data          0x00000000        0x0 obj/uc_libc_dev/stdio/stdio_uc.o
 .bss           0x00000000        0x0 obj/uc_libc_dev/stdio/stdio_uc.o
 .text.lerr_RegisterDev
                0x00000000        0xc obj/uc_libc_dev/stdio/stdio_uc.o
 .text.lputchar
                0x00000000        0xc obj/uc_libc_dev/stdio/stdio_uc.o
 .text.sformat  0x00000000       0x2a obj/uc_libc_dev/stdio/stdio_uc.o
 .text.sFormatArgs
                0x00000000       0x1c obj/uc_libc_dev/stdio/stdio_uc.o
 .text.date2str
                0x00000000       0x60 obj/uc_libc_dev/stdio/stdio_uc.o
 .text.time2str
                0x00000000       0x20 obj/uc_libc_dev/stdio/stdio_uc.o
 .rodata.str1.1
                0x00000000       0x23 obj/uc_libc_dev/stdio/stdio_uc.o
 .bss.result.4941
                0x00000000       0x40 obj/uc_libc_dev/stdio/stdio_uc.o
 .bss.result.4947
                0x00000000       0x40 obj/uc_libc_dev/stdio/stdio_uc.o
 .text          0x00000000        0x0 obj/uc_libc_dev/misc/buffer.o
 .data          0x00000000        0x0 obj/uc_libc_dev/misc/buffer.o
 .bss           0x00000000        0x0 obj/uc_libc_dev/misc/buffer.o
 .text.buffer_DumpFromFront
                0x00000000       0x42 obj/uc_libc_dev/misc/buffer.o
 .text.buffer_GetAtIndex
                0x00000000       0x1a obj/uc_libc_dev/misc/buffer.o
 .text.buffer_IsNotFull
                0x00000000       0x12 obj/uc_libc_dev/misc/buffer.o
 .text.buffer_Clear
                0x00000000        0x6 obj/uc_libc_dev/misc/buffer.o
 .text          0x00000000        0x0 obj/uc_libc_dev/misc/utils.o
 .data          0x00000000        0x0 obj/uc_libc_dev/misc/utils.o
 .bss           0x00000000        0x0 obj/uc_libc_dev/misc/utils.o
 .text.put_dump
                0x00000000       0x78 obj/uc_libc_dev/misc/utils.o
 .text.buffer_dump
                0x00000000       0x32 obj/uc_libc_dev/misc/utils.o
 .text.xatof    0x00000000      0x15c obj/uc_libc_dev/misc/utils.o
 .text.secondsToHours
                0x00000000       0x40 obj/uc_libc_dev/misc/utils.o
 .text.minutesToHours
                0x00000000       0x12 obj/uc_libc_dev/misc/utils.o
 .text.hoursToMinutes
                0x00000000        0xa obj/uc_libc_dev/misc/utils.o
 .text          0x00000000        0x0 obj/uc_libc_dev/misc/led_error.o
 .data          0x00000000        0x0 obj/uc_libc_dev/misc/led_error.o
 .bss           0x00000000        0x0 obj/uc_libc_dev/misc/led_error.o
 .text.ledError_Blink
                0x00000000       0x14 obj/uc_libc_dev/misc/led_error.o
 .text          0x00000000        0x0 obj/uc_libc_dev/keyboard/gkey.o
 .data          0x00000000        0x0 obj/uc_libc_dev/keyboard/gkey.o
 .bss           0x00000000        0x0 obj/uc_libc_dev/keyboard/gkey.o
 .text          0x00000000        0x0 obj/uc_libc_dev/sound/beep/beep.o
 .data          0x00000000        0x0 obj/uc_libc_dev/sound/beep/beep.o
 .bss           0x00000000        0x0 obj/uc_libc_dev/sound/beep/beep.o
 .text.beep_Playing
                0x00000000       0x14 obj/uc_libc_dev/sound/beep/beep.o
 .text.beep_Stop
                0x00000000       0x10 obj/uc_libc_dev/sound/beep/beep.o
 .text          0x00000000        0x0 obj/uc_libc_dev/cli/cli.o
 .data          0x00000000        0x0 obj/uc_libc_dev/cli/cli.o
 .bss           0x00000000        0x0 obj/uc_libc_dev/cli/cli.o
 .text          0x00000000        0x0 obj/uc_libc_dev/display/liquid_crystal.o
 .data          0x00000000        0x0 obj/uc_libc_dev/display/liquid_crystal.o
 .bss           0x00000000        0x0 obj/uc_libc_dev/display/liquid_crystal.o
 .text.lcd_Home
                0x00000000       0x18 obj/uc_libc_dev/display/liquid_crystal.o
 .text.lcd_NoDisplay
                0x00000000       0x18 obj/uc_libc_dev/display/liquid_crystal.o
 .text.lcd_NoCursor
                0x00000000       0x18 obj/uc_libc_dev/display/liquid_crystal.o
 .text.lcd_Cursor
                0x00000000       0x18 obj/uc_libc_dev/display/liquid_crystal.o
 .text.lcd_NoBlink
                0x00000000       0x18 obj/uc_libc_dev/display/liquid_crystal.o
 .text.lcd_Blink
                0x00000000       0x18 obj/uc_libc_dev/display/liquid_crystal.o
 .text.lcd_ScrollDisplayLeft
                0x00000000        0x6 obj/uc_libc_dev/display/liquid_crystal.o
 .text.lcd_ScrollDisplayRight
                0x00000000        0x6 obj/uc_libc_dev/display/liquid_crystal.o
 .text.lcd_LeftToRight
                0x00000000       0x18 obj/uc_libc_dev/display/liquid_crystal.o
 .text.lcd_RightToLeft
                0x00000000       0x18 obj/uc_libc_dev/display/liquid_crystal.o
 .text.lcd_AutoScroll
                0x00000000       0x18 obj/uc_libc_dev/display/liquid_crystal.o
 .text.lcd_NoAutoScroll
                0x00000000       0x18 obj/uc_libc_dev/display/liquid_crystal.o
 .text          0x00000000        0x0 obj/uc_libc_dev/display/portable/arm_lpc/lcd_drv.o
 .data          0x00000000        0x0 obj/uc_libc_dev/display/portable/arm_lpc/lcd_drv.o
 .bss           0x00000000        0x0 obj/uc_libc_dev/display/portable/arm_lpc/lcd_drv.o
 .data          0x00000000        0x0 d:/cc/arm-yagarto-5.4.2016q3/bin/../lib/gcc/arm-none-eabi/5.4.1/armv7-m\libgcc.a(_arm_addsubdf3.o)
 .bss           0x00000000        0x0 d:/cc/arm-yagarto-5.4.2016q3/bin/../lib/gcc/arm-none-eabi/5.4.1/armv7-m\libgcc.a(_arm_addsubdf3.o)
 .data          0x00000000        0x0 d:/cc/arm-yagarto-5.4.2016q3/bin/../lib/gcc/arm-none-eabi/5.4.1/armv7-m\libgcc.a(_arm_muldivdf3.o)
 .bss           0x00000000        0x0 d:/cc/arm-yagarto-5.4.2016q3/bin/../lib/gcc/arm-none-eabi/5.4.1/armv7-m\libgcc.a(_arm_muldivdf3.o)
 .data          0x00000000        0x0 d:/cc/arm-yagarto-5.4.2016q3/bin/../lib/gcc/arm-none-eabi/5.4.1/armv7-m\libgcc.a(_arm_cmpdf2.o)
 .bss           0x00000000        0x0 d:/cc/arm-yagarto-5.4.2016q3/bin/../lib/gcc/arm-none-eabi/5.4.1/armv7-m\libgcc.a(_arm_cmpdf2.o)
 .data          0x00000000        0x0 d:/cc/arm-yagarto-5.4.2016q3/bin/../lib/gcc/arm-none-eabi/5.4.1/armv7-m\libgcc.a(_arm_fixdfsi.o)
 .bss           0x00000000        0x0 d:/cc/arm-yagarto-5.4.2016q3/bin/../lib/gcc/arm-none-eabi/5.4.1/armv7-m\libgcc.a(_arm_fixdfsi.o)
 .data          0x00000000        0x0 d:/cc/arm-yagarto-5.4.2016q3/bin/../lib/gcc/arm-none-eabi/5.4.1/armv7-m\libgcc.a(_arm_addsubsf3.o)
 .bss           0x00000000        0x0 d:/cc/arm-yagarto-5.4.2016q3/bin/../lib/gcc/arm-none-eabi/5.4.1/armv7-m\libgcc.a(_arm_addsubsf3.o)
 .data          0x00000000        0x0 d:/cc/arm-yagarto-5.4.2016q3/bin/../lib/gcc/arm-none-eabi/5.4.1/armv7-m\libgcc.a(_arm_muldivsf3.o)
 .bss           0x00000000        0x0 d:/cc/arm-yagarto-5.4.2016q3/bin/../lib/gcc/arm-none-eabi/5.4.1/armv7-m\libgcc.a(_arm_muldivsf3.o)
 .text          0x00000000        0x0 d:/cc/arm-yagarto-5.4.2016q3/bin/../lib/gcc/arm-none-eabi/5.4.1/../../../../arm-none-eabi/lib/armv7-m\libc.a(lib_a-locale.o)
 .data          0x00000000        0x0 d:/cc/arm-yagarto-5.4.2016q3/bin/../lib/gcc/arm-none-eabi/5.4.1/../../../../arm-none-eabi/lib/armv7-m\libc.a(lib_a-locale.o)
 .bss           0x00000000        0x0 d:/cc/arm-yagarto-5.4.2016q3/bin/../lib/gcc/arm-none-eabi/5.4.1/../../../../arm-none-eabi/lib/armv7-m\libc.a(lib_a-locale.o)
 .text._setlocale_r
                0x00000000       0x40 d:/cc/arm-yagarto-5.4.2016q3/bin/../lib/gcc/arm-none-eabi/5.4.1/../../../../arm-none-eabi/lib/armv7-m\libc.a(lib_a-locale.o)
 .text.__locale_mb_cur_max
                0x00000000       0x1c d:/cc/arm-yagarto-5.4.2016q3/bin/../lib/gcc/arm-none-eabi/5.4.1/../../../../arm-none-eabi/lib/armv7-m\libc.a(lib_a-locale.o)
 .text.__locale_ctype_ptr_l
                0x00000000        0x8 d:/cc/arm-yagarto-5.4.2016q3/bin/../lib/gcc/arm-none-eabi/5.4.1/../../../../arm-none-eabi/lib/armv7-m\libc.a(lib_a-locale.o)
 .text.setlocale
                0x00000000       0x10 d:/cc/arm-yagarto-5.4.2016q3/bin/../lib/gcc/arm-none-eabi/5.4.1/../../../../arm-none-eabi/lib/armv7-m\libc.a(lib_a-locale.o)
 .bss._PathLocale
                0x00000000        0x4 d:/cc/arm-yagarto-5.4.2016q3/bin/../lib/gcc/arm-none-eabi/5.4.1/../../../../arm-none-eabi/lib/armv7-m\libc.a(lib_a-locale.o)
 .text          0x00000000        0x0 d:/cc/arm-yagarto-5.4.2016q3/bin/../lib/gcc/arm-none-eabi/5.4.1/../../../../arm-none-eabi/lib/armv7-m\libc.a(lib_a-mbtowc_r.o)
 .data          0x00000000        0x0 d:/cc/arm-yagarto-5.4.2016q3/bin/../lib/gcc/arm-none-eabi/5.4.1/../../../../arm-none-eabi/lib/armv7-m\libc.a(lib_a-mbtowc_r.o)
 .bss           0x00000000        0x0 d:/cc/arm-yagarto-5.4.2016q3/bin/../lib/gcc/arm-none-eabi/5.4.1/../../../../arm-none-eabi/lib/armv7-m\libc.a(lib_a-mbtowc_r.o)
 .text._mbtowc_r
                0x00000000       0x24 d:/cc/arm-yagarto-5.4.2016q3/bin/../lib/gcc/arm-none-eabi/5.4.1/../../../../arm-none-eabi/lib/armv7-m\libc.a(lib_a-mbtowc_r.o)
 .text          0x00000000        0x0 d:/cc/arm-yagarto-5.4.2016q3/bin/../lib/gcc/arm-none-eabi/5.4.1/../../../../arm-none-eabi/lib/armv7-m\libc.a(lib_a-memset.o)
 .data          0x00000000        0x0 d:/cc/arm-yagarto-5.4.2016q3/bin/../lib/gcc/arm-none-eabi/5.4.1/../../../../arm-none-eabi/lib/armv7-m\libc.a(lib_a-memset.o)
 .bss           0x00000000        0x0 d:/cc/arm-yagarto-5.4.2016q3/bin/../lib/gcc/arm-none-eabi/5.4.1/../../../../arm-none-eabi/lib/armv7-m\libc.a(lib_a-memset.o)
 .data          0x00000000        0x0 d:/cc/arm-yagarto-5.4.2016q3/bin/../lib/gcc/arm-none-eabi/5.4.1/../../../../arm-none-eabi/lib/armv7-m\libc.a(lib_a-strcmp.o)
 .bss           0x00000000        0x0 d:/cc/arm-yagarto-5.4.2016q3/bin/../lib/gcc/arm-none-eabi/5.4.1/../../../../arm-none-eabi/lib/armv7-m\libc.a(lib_a-strcmp.o)
 .text          0x00000000        0x0 d:/cc/arm-yagarto-5.4.2016q3/bin/../lib/gcc/arm-none-eabi/5.4.1/../../../../arm-none-eabi/lib/armv7-m\libc.a(lib_a-strlen-stub.o)
 .data          0x00000000        0x0 d:/cc/arm-yagarto-5.4.2016q3/bin/../lib/gcc/arm-none-eabi/5.4.1/../../../../arm-none-eabi/lib/armv7-m\libc.a(lib_a-strlen-stub.o)
 .bss           0x00000000        0x0 d:/cc/arm-yagarto-5.4.2016q3/bin/../lib/gcc/arm-none-eabi/5.4.1/../../../../arm-none-eabi/lib/armv7-m\libc.a(lib_a-strlen-stub.o)
 .text          0x00000000        0x0 d:/cc/arm-yagarto-5.4.2016q3/bin/../lib/gcc/arm-none-eabi/5.4.1/../../../../arm-none-eabi/lib/armv7-m\libc.a(lib_a-wctomb_r.o)
 .data          0x00000000        0x0 d:/cc/arm-yagarto-5.4.2016q3/bin/../lib/gcc/arm-none-eabi/5.4.1/../../../../arm-none-eabi/lib/armv7-m\libc.a(lib_a-wctomb_r.o)
 .bss           0x00000000        0x0 d:/cc/arm-yagarto-5.4.2016q3/bin/../lib/gcc/arm-none-eabi/5.4.1/../../../../arm-none-eabi/lib/armv7-m\libc.a(lib_a-wctomb_r.o)
 .text._wctomb_r
                0x00000000       0x24 d:/cc/arm-yagarto-5.4.2016q3/bin/../lib/gcc/arm-none-eabi/5.4.1/../../../../arm-none-eabi/lib/armv7-m\libc.a(lib_a-wctomb_r.o)
 .text          0x00000000        0x0 d:/cc/arm-yagarto-5.4.2016q3/bin/../lib/gcc/arm-none-eabi/5.4.1/../../../../arm-none-eabi/lib/armv7-m\libc.a(lib_a-ctype_.o)
 .data          0x00000000        0x0 d:/cc/arm-yagarto-5.4.2016q3/bin/../lib/gcc/arm-none-eabi/5.4.1/../../../../arm-none-eabi/lib/armv7-m\libc.a(lib_a-ctype_.o)
 .bss           0x00000000        0x0 d:/cc/arm-yagarto-5.4.2016q3/bin/../lib/gcc/arm-none-eabi/5.4.1/../../../../arm-none-eabi/lib/armv7-m\libc.a(lib_a-ctype_.o)
 .text          0x00000000        0x0 d:/cc/arm-yagarto-5.4.2016q3/bin/../lib/gcc/arm-none-eabi/5.4.1/../../../../arm-none-eabi/lib/armv7-m\libc.a(lib_a-impure.o)
 .data          0x00000000        0x0 d:/cc/arm-yagarto-5.4.2016q3/bin/../lib/gcc/arm-none-eabi/5.4.1/../../../../arm-none-eabi/lib/armv7-m\libc.a(lib_a-impure.o)
 .bss           0x00000000        0x0 d:/cc/arm-yagarto-5.4.2016q3/bin/../lib/gcc/arm-none-eabi/5.4.1/../../../../arm-none-eabi/lib/armv7-m\libc.a(lib_a-impure.o)
 .rodata._global_impure_ptr
                0x00000000        0x4 d:/cc/arm-yagarto-5.4.2016q3/bin/../lib/gcc/arm-none-eabi/5.4.1/../../../../arm-none-eabi/lib/armv7-m\libc.a(lib_a-impure.o)

Memory Configuration

Name             Origin             Length             Attributes
FLASH            0x00000000         0x00010000         xr
RAM              0x10000000         0x00004000         rw
*default*        0x00000000         0xffffffff

Linker script and memory map

LOAD obj/uc_libc_dev/_arch/arm_lpc/common/arm.o
LOAD obj/uc_libc_dev/_arch/arm_lpc/common/startup/startup.o
LOAD obj/uc_libc_dev/_arch/arm_lpc/common/vic_cortexm3.o
LOAD obj/uc_libc_dev/_arch/arm_lpc/timer/systick.o
LOAD obj/uc_libc_dev/_arch/arm_lpc/timer/delay.o
LOAD obj/uc_libc_dev/_arch/arm_lpc/uart/uart0_irq.o
LOAD obj/main.o
LOAD obj/app.o
LOAD obj/prompt.o
LOAD obj/uc_libc_dev/stdio/stdio_uc.o
LOAD obj/uc_libc_dev/misc/buffer.o
LOAD obj/uc_libc_dev/misc/utils.o
LOAD obj/uc_libc_dev/misc/led_error.o
LOAD obj/uc_libc_dev/keyboard/gkey.o
LOAD obj/uc_libc_dev/sound/beep/beep.o
LOAD obj/uc_libc_dev/cli/cli.o
LOAD obj/uc_libc_dev/display/liquid_crystal.o
LOAD obj/uc_libc_dev/display/portable/arm_lpc/lcd_drv.o
LOAD d:/cc/arm-yagarto-5.4.2016q3/bin/../lib/gcc/arm-none-eabi/5.4.1/../../../../arm-none-eabi/lib/armv7-m\libm.a
LOAD d:/cc/arm-yagarto-5.4.2016q3/bin/../lib/gcc/arm-none-eabi/5.4.1/armv7-m\libgcc.a
LOAD d:/cc/arm-yagarto-5.4.2016q3/bin/../lib/gcc/arm-none-eabi/5.4.1/../../../../arm-none-eabi/lib/armv7-m\libc.a
                0x10004000                _stack = (ORIGIN (RAM) + LENGTH (RAM))

.text           0x00000000     0x1268
 CREATE_OBJECT_SYMBOLS
 *(.vectors)
 .vectors       0x00000000       0xe4 obj/uc_libc_dev/_arch/arm_lpc/common/vic_cortexm3.o
                0x00000000                gVectors
                0x000002fc                . = 0x2fc
 *fill*         0x000000e4      0x218 
 *(.crp)
 *startup.o(.text)
 *(.text)
 .text          0x000002fc      0x370 d:/cc/arm-yagarto-5.4.2016q3/bin/../lib/gcc/arm-none-eabi/5.4.1/armv7-m\libgcc.a(_arm_addsubdf3.o)
                0x000002fc                __aeabi_drsub
                0x00000304                __aeabi_dsub
                0x00000304                __subdf3
                0x00000308                __aeabi_dadd
                0x00000308                __adddf3
                0x00000580                __floatunsidf
                0x00000580                __aeabi_ui2d
                0x000005a0                __floatsidf
                0x000005a0                __aeabi_i2d
                0x000005c4                __aeabi_f2d
                0x000005c4                __extendsfdf2
                0x00000600                __floatundidf
                0x00000600                __aeabi_ul2d
                0x00000610                __floatdidf
                0x00000610                __aeabi_l2d
 .text          0x0000066c      0x424 d:/cc/arm-yagarto-5.4.2016q3/bin/../lib/gcc/arm-none-eabi/5.4.1/armv7-m\libgcc.a(_arm_muldivdf3.o)
                0x0000066c                __aeabi_dmul
                0x0000066c                __muldf3
                0x000008c0                __divdf3
                0x000008c0                __aeabi_ddiv
 .text          0x00000a90      0x110 d:/cc/arm-yagarto-5.4.2016q3/bin/../lib/gcc/arm-none-eabi/5.4.1/armv7-m\libgcc.a(_arm_cmpdf2.o)
                0x00000a90                __gtdf2
                0x00000a90                __gedf2
                0x00000a98                __ltdf2
                0x00000a98                __ledf2
                0x00000aa0                __nedf2
                0x00000aa0                __eqdf2
                0x00000aa0                __cmpdf2
                0x00000b1c                __aeabi_cdrcmple
                0x00000b2c                __aeabi_cdcmpeq
                0x00000b2c                __aeabi_cdcmple
                0x00000b3c                __aeabi_dcmpeq
                0x00000b50                __aeabi_dcmplt
                0x00000b64                __aeabi_dcmple
                0x00000b78                __aeabi_dcmpge
                0x00000b8c                __aeabi_dcmpgt
 .text          0x00000ba0       0x50 d:/cc/arm-yagarto-5.4.2016q3/bin/../lib/gcc/arm-none-eabi/5.4.1/armv7-m\libgcc.a(_arm_fixdfsi.o)
                0x00000ba0                __aeabi_d2iz
                0x00000ba0                __fixdfsi
 .text          0x00000bf0      0x21c d:/cc/arm-yagarto-5.4.2016q3/bin/../lib/gcc/arm-none-eabi/5.4.1/armv7-m\libgcc.a(_arm_addsubsf3.o)
                0x00000bf0                __aeabi_frsub
                0x00000bf8                __subsf3
                0x00000bf8                __aeabi_fsub
                0x00000bfc                __aeabi_fadd
                0x00000bfc                __addsf3
                0x00000d5c                __aeabi_ui2f
                0x00000d5c                __floatunsisf
                0x00000d64                __aeabi_i2f
                0x00000d64                __floatsisf
                0x00000d80                __aeabi_ul2f
                0x00000d80                __floatundisf
                0x00000d90                __aeabi_l2f
                0x00000d90                __floatdisf
 .text          0x00000e0c      0x2a0 d:/cc/arm-yagarto-5.4.2016q3/bin/../lib/gcc/arm-none-eabi/5.4.1/armv7-m\libgcc.a(_arm_muldivsf3.o)
                0x00000e0c                __mulsf3
                0x00000e0c                __aeabi_fmul
                0x00000f74                __aeabi_fdiv
                0x00000f74                __divsf3
 .text          0x000010ac      0x1bc d:/cc/arm-yagarto-5.4.2016q3/bin/../lib/gcc/arm-none-eabi/5.4.1/../../../../arm-none-eabi/lib/armv7-m\libc.a(lib_a-strcmp.o)
                0x000010ac                strcmp
 *(.glue_7)
 .glue_7        0x00001268        0x0 linker stubs
 *(.glue_7t)
 .glue_7t       0x00001268        0x0 linker stubs

.vfp11_veneer   0x00001268        0x0
 .vfp11_veneer  0x00001268        0x0 linker stubs

.v4_bx          0x00001268        0x0
 .v4_bx         0x00001268        0x0 linker stubs

.text.arm_Init  0x00001268      0x138
 .text.arm_Init
                0x00001268      0x138 obj/uc_libc_dev/_arch/arm_lpc/common/arm.o
                0x00001268                arm_Init

.iplt           0x000013a0        0x0
 .iplt          0x000013a0        0x0 obj/uc_libc_dev/_arch/arm_lpc/common/arm.o

.text._start    0x000013a0       0x48
 .text._start   0x000013a0       0x48 obj/uc_libc_dev/_arch/arm_lpc/common/startup/startup.o
                0x000013a0                _start

.text.nmi_ISR   0x000013e8       0x20
 .text.nmi_ISR  0x000013e8       0x20 obj/uc_libc_dev/_arch/arm_lpc/common/vic_cortexm3.o
                0x000013e8                nmi_ISR

.text.hardFault_ISR
                0x00001408       0x50
 .text.hardFault_ISR
                0x00001408       0x50 obj/uc_libc_dev/_arch/arm_lpc/common/vic_cortexm3.o
                0x00001408                hardFault_ISR

.text.memManage_ISR
                0x00001458       0x20
 .text.memManage_ISR
                0x00001458       0x20 obj/uc_libc_dev/_arch/arm_lpc/common/vic_cortexm3.o
                0x00001458                memManage_ISR

.text.busFault_ISR
                0x00001478       0x20
 .text.busFault_ISR
                0x00001478       0x20 obj/uc_libc_dev/_arch/arm_lpc/common/vic_cortexm3.o
                0x00001478                busFault_ISR

.text.usageFault_ISR
                0x00001498       0x20
 .text.usageFault_ISR
                0x00001498       0x20 obj/uc_libc_dev/_arch/arm_lpc/common/vic_cortexm3.o
                0x00001498                usageFault_ISR

.text.svc_ISR   0x000014b8       0x20
 .text.svc_ISR  0x000014b8       0x20 obj/uc_libc_dev/_arch/arm_lpc/common/vic_cortexm3.o
                0x000014b8                svc_ISR

.text.debugMon_ISR
                0x000014d8       0x20
 .text.debugMon_ISR
                0x000014d8       0x20 obj/uc_libc_dev/_arch/arm_lpc/common/vic_cortexm3.o
                0x000014d8                debugMon_ISR

.text.pendSV_ISR
                0x000014f8       0x20
 .text.pendSV_ISR
                0x000014f8       0x20 obj/uc_libc_dev/_arch/arm_lpc/common/vic_cortexm3.o
                0x000014f8                pendSV_ISR

.text.wdt_ISR   0x00001518       0x20
 .text.wdt_ISR  0x00001518       0x20 obj/uc_libc_dev/_arch/arm_lpc/common/vic_cortexm3.o
                0x00001518                wdt_ISR

.text.timer0_ISR
                0x00001538       0x20
 .text.timer0_ISR
                0x00001538       0x20 obj/uc_libc_dev/_arch/arm_lpc/common/vic_cortexm3.o
                0x00001538                timer0_ISR

.text.timer1_ISR
                0x00001558       0x20
 .text.timer1_ISR
                0x00001558       0x20 obj/uc_libc_dev/_arch/arm_lpc/common/vic_cortexm3.o
                0x00001558                timer1_ISR

.text.timer2_ISR
                0x00001578       0x20
 .text.timer2_ISR
                0x00001578       0x20 obj/uc_libc_dev/_arch/arm_lpc/common/vic_cortexm3.o
                0x00001578                timer2_ISR

.text.timer3_ISR
                0x00001598       0x20
 .text.timer3_ISR
                0x00001598       0x20 obj/uc_libc_dev/_arch/arm_lpc/common/vic_cortexm3.o
                0x00001598                timer3_ISR

.text.uart1_ISR
                0x000015b8       0x20
 .text.uart1_ISR
                0x000015b8       0x20 obj/uc_libc_dev/_arch/arm_lpc/common/vic_cortexm3.o
                0x000015b8                uart1_ISR

.text.uart2_ISR
                0x000015d8       0x20
 .text.uart2_ISR
                0x000015d8       0x20 obj/uc_libc_dev/_arch/arm_lpc/common/vic_cortexm3.o
                0x000015d8                uart2_ISR

.text.uart3_ISR
                0x000015f8       0x20
 .text.uart3_ISR
                0x000015f8       0x20 obj/uc_libc_dev/_arch/arm_lpc/common/vic_cortexm3.o
                0x000015f8                uart3_ISR

.text.pwm_ISR   0x00001618       0x20
 .text.pwm_ISR  0x00001618       0x20 obj/uc_libc_dev/_arch/arm_lpc/common/vic_cortexm3.o
                0x00001618                pwm_ISR

.text.i2c0_ISR  0x00001638       0x20
 .text.i2c0_ISR
                0x00001638       0x20 obj/uc_libc_dev/_arch/arm_lpc/common/vic_cortexm3.o
                0x00001638                i2c0_ISR

.text.i2c1_ISR  0x00001658       0x20
 .text.i2c1_ISR
                0x00001658       0x20 obj/uc_libc_dev/_arch/arm_lpc/common/vic_cortexm3.o
                0x00001658                i2c1_ISR

.text.i2c2_ISR  0x00001678       0x20
 .text.i2c2_ISR
                0x00001678       0x20 obj/uc_libc_dev/_arch/arm_lpc/common/vic_cortexm3.o
                0x00001678                i2c2_ISR

.text.spi_ISR   0x00001698       0x20
 .text.spi_ISR  0x00001698       0x20 obj/uc_libc_dev/_arch/arm_lpc/common/vic_cortexm3.o
                0x00001698                spi_ISR

.text.ssp0_ISR  0x000016b8       0x20
 .text.ssp0_ISR
                0x000016b8       0x20 obj/uc_libc_dev/_arch/arm_lpc/common/vic_cortexm3.o
                0x000016b8                ssp0_ISR

.text.ssp1_ISR  0x000016d8       0x20
 .text.ssp1_ISR
                0x000016d8       0x20 obj/uc_libc_dev/_arch/arm_lpc/common/vic_cortexm3.o
                0x000016d8                ssp1_ISR

.text.pll0_ISR  0x000016f8       0x20
 .text.pll0_ISR
                0x000016f8       0x20 obj/uc_libc_dev/_arch/arm_lpc/common/vic_cortexm3.o
                0x000016f8                pll0_ISR

.text.rtc_ISR   0x00001718       0x20
 .text.rtc_ISR  0x00001718       0x20 obj/uc_libc_dev/_arch/arm_lpc/common/vic_cortexm3.o
                0x00001718                rtc_ISR

.text.eint0_ISR
                0x00001738       0x20
 .text.eint0_ISR
                0x00001738       0x20 obj/uc_libc_dev/_arch/arm_lpc/common/vic_cortexm3.o
                0x00001738                eint0_ISR

.text.eint1_ISR
                0x00001758       0x20
 .text.eint1_ISR
                0x00001758       0x20 obj/uc_libc_dev/_arch/arm_lpc/common/vic_cortexm3.o
                0x00001758                eint1_ISR

.text.eint2_ISR
                0x00001778       0x20
 .text.eint2_ISR
                0x00001778       0x20 obj/uc_libc_dev/_arch/arm_lpc/common/vic_cortexm3.o
                0x00001778                eint2_ISR

.text.eint3_ISR
                0x00001798       0x20
 .text.eint3_ISR
                0x00001798       0x20 obj/uc_libc_dev/_arch/arm_lpc/common/vic_cortexm3.o
                0x00001798                eint3_ISR

.text.adc_ISR   0x000017b8       0x20
 .text.adc_ISR  0x000017b8       0x20 obj/uc_libc_dev/_arch/arm_lpc/common/vic_cortexm3.o
                0x000017b8                adc_ISR

.text.bod_ISR   0x000017d8       0x20
 .text.bod_ISR  0x000017d8       0x20 obj/uc_libc_dev/_arch/arm_lpc/common/vic_cortexm3.o
                0x000017d8                bod_ISR

.text.usbHost_ISR
                0x000017f8       0x20
 .text.usbHost_ISR
                0x000017f8       0x20 obj/uc_libc_dev/_arch/arm_lpc/common/vic_cortexm3.o
                0x000017f8                usbHost_ISR

.text.can_ISR   0x00001818       0x20
 .text.can_ISR  0x00001818       0x20 obj/uc_libc_dev/_arch/arm_lpc/common/vic_cortexm3.o
                0x00001818                can_ISR

.text.dma_ISR   0x00001838       0x20
 .text.dma_ISR  0x00001838       0x20 obj/uc_libc_dev/_arch/arm_lpc/common/vic_cortexm3.o
                0x00001838                dma_ISR

.text.i2s_ISR   0x00001858       0x20
 .text.i2s_ISR  0x00001858       0x20 obj/uc_libc_dev/_arch/arm_lpc/common/vic_cortexm3.o
                0x00001858                i2s_ISR

.text.enet_ISR  0x00001878       0x20
 .text.enet_ISR
                0x00001878       0x20 obj/uc_libc_dev/_arch/arm_lpc/common/vic_cortexm3.o
                0x00001878                enet_ISR

.text.rit_ISR   0x00001898       0x20
 .text.rit_ISR  0x00001898       0x20 obj/uc_libc_dev/_arch/arm_lpc/common/vic_cortexm3.o
                0x00001898                rit_ISR

.text.mcpwm_ISR
                0x000018b8       0x20
 .text.mcpwm_ISR
                0x000018b8       0x20 obj/uc_libc_dev/_arch/arm_lpc/common/vic_cortexm3.o
                0x000018b8                mcpwm_ISR

.text.qei_ISR   0x000018d8       0x20
 .text.qei_ISR  0x000018d8       0x20 obj/uc_libc_dev/_arch/arm_lpc/common/vic_cortexm3.o
                0x000018d8                qei_ISR

.text.pll1_ISR  0x000018f8       0x20
 .text.pll1_ISR
                0x000018f8       0x20 obj/uc_libc_dev/_arch/arm_lpc/common/vic_cortexm3.o
                0x000018f8                pll1_ISR

.text.usbAct_ISR
                0x00001918       0x20
 .text.usbAct_ISR
                0x00001918       0x20 obj/uc_libc_dev/_arch/arm_lpc/common/vic_cortexm3.o
                0x00001918                usbAct_ISR

.text.canAct_ISR
                0x00001938       0x20
 .text.canAct_ISR
                0x00001938       0x20 obj/uc_libc_dev/_arch/arm_lpc/common/vic_cortexm3.o
                0x00001938                canAct_ISR

.text.uart4_ISR
                0x00001958       0x20
 .text.uart4_ISR
                0x00001958       0x20 obj/uc_libc_dev/_arch/arm_lpc/common/vic_cortexm3.o
                0x00001958                uart4_ISR

.text.ssp2_ISR  0x00001978       0x20
 .text.ssp2_ISR
                0x00001978       0x20 obj/uc_libc_dev/_arch/arm_lpc/common/vic_cortexm3.o
                0x00001978                ssp2_ISR

.text.lcd_ISR   0x00001998       0x20
 .text.lcd_ISR  0x00001998       0x20 obj/uc_libc_dev/_arch/arm_lpc/common/vic_cortexm3.o
                0x00001998                lcd_ISR

.text.gpio_ISR  0x000019b8       0x20
 .text.gpio_ISR
                0x000019b8       0x20 obj/uc_libc_dev/_arch/arm_lpc/common/vic_cortexm3.o
                0x000019b8                gpio_ISR

.text.pwm0_ISR  0x000019d8       0x20
 .text.pwm0_ISR
                0x000019d8       0x20 obj/uc_libc_dev/_arch/arm_lpc/common/vic_cortexm3.o
                0x000019d8                pwm0_ISR

.text.eeprom_ISR
                0x000019f8       0x20
 .text.eeprom_ISR
                0x000019f8       0x20 obj/uc_libc_dev/_arch/arm_lpc/common/vic_cortexm3.o
                0x000019f8                eeprom_ISR

.text.nvic_setPendingIRQ
                0x00001a18       0x1a
 .text.nvic_setPendingIRQ
                0x00001a18       0x1a obj/uc_libc_dev/_arch/arm_lpc/common/vic_cortexm3.o
                0x00001a18                nvic_setPendingIRQ

.text.nvic_enableIRQ
                0x00001a32        0x4
 .text.nvic_enableIRQ
                0x00001a32        0x4 obj/uc_libc_dev/_arch/arm_lpc/common/vic_cortexm3.o
                0x00001a32                nvic_enableIRQ

.text.nvic_clearPendingIRQ
                0x00001a38       0x18
 .text.nvic_clearPendingIRQ
                0x00001a38       0x18 obj/uc_libc_dev/_arch/arm_lpc/common/vic_cortexm3.o
                0x00001a38                nvic_clearPendingIRQ

.text.nvic_setPriority
                0x00001a50       0x44
 .text.nvic_setPriority
                0x00001a50       0x44 obj/uc_libc_dev/_arch/arm_lpc/common/vic_cortexm3.o
                0x00001a50                nvic_setPriority

.text.nvic_SetIntHandler
                0x00001a94        0xc
 .text.nvic_SetIntHandler
                0x00001a94        0xc obj/uc_libc_dev/_arch/arm_lpc/common/vic_cortexm3.o
                0x00001a94                nvic_SetIntHandler

.text.systime_Init
                0x00001aa0       0x5c
 .text.systime_Init
                0x00001aa0       0x5c obj/uc_libc_dev/_arch/arm_lpc/timer/systick.o
                0x00001aa0                systime_Init

.text.systime_SetIntHandler
                0x00001afc       0x14
 .text.systime_SetIntHandler
                0x00001afc       0x14 obj/uc_libc_dev/_arch/arm_lpc/timer/systick.o
                0x00001afc                systime_SetIntHandler

.text.sysTick_ISR
                0x00001b10       0x64
 .text.sysTick_ISR
                0x00001b10       0x64 obj/uc_libc_dev/_arch/arm_lpc/timer/systick.o
                0x00001b10                sysTick_ISR

.text.delay     0x00001b74        0x6
 .text.delay    0x00001b74        0x6 obj/uc_libc_dev/_arch/arm_lpc/timer/delay.o
                0x00001b74                delay

.text.uart0_SetBaudrate
                0x00001b80       0xec
 .text.uart0_SetBaudrate
                0x00001b80       0xec obj/uc_libc_dev/_arch/arm_lpc/uart/uart0_irq.o
                0x00001b80                uart0_SetBaudrate

.text.uart0_Init
                0x00001c6c       0xb0
 .text.uart0_Init
                0x00001c6c       0xb0 obj/uc_libc_dev/_arch/arm_lpc/uart/uart0_irq.o
                0x00001c6c                uart0_Init

.text.uart0_GetChar
                0x00001d1c       0x44
 .text.uart0_GetChar
                0x00001d1c       0x44 obj/uc_libc_dev/_arch/arm_lpc/uart/uart0_irq.o
                0x00001d1c                uart0_GetChar

.text.uart0_PutChar
                0x00001d60       0x68
 .text.uart0_PutChar
                0x00001d60       0x68 obj/uc_libc_dev/_arch/arm_lpc/uart/uart0_irq.o
                0x00001d60                uart0_PutChar

.text.uart0_BasicPutChar
                0x00001dc8       0x1c
 .text.uart0_BasicPutChar
                0x00001dc8       0x1c obj/uc_libc_dev/_arch/arm_lpc/uart/uart0_irq.o
                0x00001dc8                uart0_BasicPutChar

.text.uart0_ISR
                0x00001de4       0xb4
 .text.uart0_ISR
                0x00001de4       0xb4 obj/uc_libc_dev/_arch/arm_lpc/uart/uart0_irq.o
                0x00001de4                uart0_ISR

.text.showVicError
                0x00001e98       0x78
 .text.showVicError
                0x00001e98       0x78 obj/main.o

.text.startup.main
                0x00001f10       0xc0
 .text.startup.main
                0x00001f10       0xc0 obj/main.o
                0x00001f10                main

.text.onKeyDown
                0x00001fd0       0x34
 .text.onKeyDown
                0x00001fd0       0x34 obj/app.o
                0x00001fd0                onKeyDown

.text.onKeyPress
                0x00002004       0x18
 .text.onKeyPress
                0x00002004       0x18 obj/app.o
                0x00002004                onKeyPress

.text.onKeyUp   0x0000201c       0x18
 .text.onKeyUp  0x0000201c       0x18 obj/app.o
                0x0000201c                onKeyUp

.text.relay_Init
                0x00002034       0x28
 .text.relay_Init
                0x00002034       0x28 obj/app.o
                0x00002034                relay_Init

.text.relay_Set
                0x0000205c       0x30
 .text.relay_Set
                0x0000205c       0x30 obj/app.o
                0x0000205c                relay_Set

.text.relay_Tick
                0x0000208c       0x68
 .text.relay_Tick
                0x0000208c       0x68 obj/app.o
                0x0000208c                relay_Tick

.text.app_Init  0x000020f4      0x12c
 .text.app_Init
                0x000020f4      0x12c obj/app.o
                0x000020f4                app_Init

.text.app_Tick  0x00002220       0xa4
 .text.app_Tick
                0x00002220       0xa4 obj/app.o
                0x00002220                app_Tick

.text.app_Process
                0x000022c4       0xc8
 .text.app_Process
                0x000022c4       0xc8 obj/app.o
                0x000022c4                app_Process

.text.prompt_ClearTicks
                0x0000238c       0x10
 .text.prompt_ClearTicks
                0x0000238c       0x10 obj/prompt.o

.text.prompt_STS
                0x0000239c       0x6c
 .text.prompt_STS
                0x0000239c       0x6c obj/prompt.o

.text.prompt_Dump
                0x00002408       0x8a
 .text.prompt_Dump
                0x00002408       0x8a obj/prompt.o

.text.prompt_Beep
                0x00002492       0x1a
 .text.prompt_Beep
                0x00002492       0x1a obj/prompt.o

.text.prompt_Relay
                0x000024ac       0x68
 .text.prompt_Relay
                0x000024ac       0x68 obj/prompt.o

.text.prompt_Process
                0x00002514       0x88
 .text.prompt_Process
                0x00002514       0x88 obj/prompt.o
                0x00002514                prompt_Process

.text.print_putchar
                0x0000259c       0x74
 .text.print_putchar
                0x0000259c       0x74 obj/uc_libc_dev/stdio/stdio_uc.o

.text.print_fill
                0x00002610       0x1a
 .text.print_fill
                0x00002610       0x1a obj/uc_libc_dev/stdio/stdio_uc.o

.text.print_int
                0x0000262a       0x58
 .text.print_int
                0x0000262a       0x58 obj/uc_libc_dev/stdio/stdio_uc.o

.text.print_long
                0x00002682       0x4e
 .text.print_long
                0x00002682       0x4e obj/uc_libc_dev/stdio/stdio_uc.o

.text.print_float
                0x000026d0       0xb4
 .text.print_float
                0x000026d0       0xb4 obj/uc_libc_dev/stdio/stdio_uc.o

.text.rprintf_RegisterDev
                0x00002784       0x30
 .text.rprintf_RegisterDev
                0x00002784       0x30 obj/uc_libc_dev/stdio/stdio_uc.o
                0x00002784                rprintf_RegisterDev

.text.lputchar_RegisterDev
                0x000027b4        0xc
 .text.lputchar_RegisterDev
                0x000027b4        0xc obj/uc_libc_dev/stdio/stdio_uc.o
                0x000027b4                lputchar_RegisterDev

.text.ldebug_RegisterDev
                0x000027c0        0xc
 .text.ldebug_RegisterDev
                0x000027c0        0xc obj/uc_libc_dev/stdio/stdio_uc.o
                0x000027c0                ldebug_RegisterDev

.text.lgetchar_RegisterDev
                0x000027cc        0xc
 .text.lgetchar_RegisterDev
                0x000027cc        0xc obj/uc_libc_dev/stdio/stdio_uc.o
                0x000027cc                lgetchar_RegisterDev

.text.doprint   0x000027d8      0x378
 .text.doprint  0x000027d8      0x378 obj/uc_libc_dev/stdio/stdio_uc.o
                0x000027d8                doprint

.text.lgetchar  0x00002b50        0xc
 .text.lgetchar
                0x00002b50        0xc obj/uc_libc_dev/stdio/stdio_uc.o
                0x00002b50                lgetchar

.text.rprintf   0x00002b5c       0x2a
 .text.rprintf  0x00002b5c       0x2a obj/uc_libc_dev/stdio/stdio_uc.o
                0x00002b5c                rprintf

.text.buffer_Init
                0x00002b86        0xc
 .text.buffer_Init
                0x00002b86        0xc obj/uc_libc_dev/misc/buffer.o
                0x00002b86                buffer_Init

.text.buffer_GetFromFront
                0x00002b92       0x44
 .text.buffer_GetFromFront
                0x00002b92       0x44 obj/uc_libc_dev/misc/buffer.o
                0x00002b92                buffer_GetFromFront

.text.buffer_AddToEnd
                0x00002bd6       0x3a
 .text.buffer_AddToEnd
                0x00002bd6       0x3a obj/uc_libc_dev/misc/buffer.o
                0x00002bd6                buffer_AddToEnd

.text.buffer_IsEmpty
                0x00002c10        0xc
 .text.buffer_IsEmpty
                0x00002c10        0xc obj/uc_libc_dev/misc/buffer.o
                0x00002c10                buffer_IsEmpty

.text.put_dump16
                0x00002c1c       0x94
 .text.put_dump16
                0x00002c1c       0x94 obj/uc_libc_dev/misc/utils.o
                0x00002c1c                put_dump16

.text.xatoi     0x00002cb0       0xa8
 .text.xatoi    0x00002cb0       0xa8 obj/uc_libc_dev/misc/utils.o
                0x00002cb0                xatoi

.text.ledError_Init
                0x00002d58       0x18
 .text.ledError_Init
                0x00002d58       0x18 obj/uc_libc_dev/misc/led_error.o
                0x00002d58                ledError_Init

.text.ledError_Tick
                0x00002d70       0x90
 .text.ledError_Tick
                0x00002d70       0x90 obj/uc_libc_dev/misc/led_error.o
                0x00002d70                ledError_Tick

.text.gKey_Init
                0x00002e00       0x24
 .text.gKey_Init
                0x00002e00       0x24 obj/uc_libc_dev/keyboard/gkey.o
                0x00002e00                gKey_Init

.text.gKey_Tick
                0x00002e24       0x14
 .text.gKey_Tick
                0x00002e24       0x14 obj/uc_libc_dev/keyboard/gkey.o
                0x00002e24                gKey_Tick

.text.gKey_Process
                0x00002e38       0xa8
 .text.gKey_Process
                0x00002e38       0xa8 obj/uc_libc_dev/keyboard/gkey.o
                0x00002e38                gKey_Process

.text.beep_SetType
                0x00002ee0       0xa0
 .text.beep_SetType
                0x00002ee0       0xa0 obj/uc_libc_dev/sound/beep/beep.o

.text.beep_Init
                0x00002f80       0x2c
 .text.beep_Init
                0x00002f80       0x2c obj/uc_libc_dev/sound/beep/beep.o
                0x00002f80                beep_Init

.text.beep_Play
                0x00002fac       0x24
 .text.beep_Play
                0x00002fac       0x24 obj/uc_libc_dev/sound/beep/beep.o
                0x00002fac                beep_Play

.text.beep_Tick
                0x00002fd0       0x8c
 .text.beep_Tick
                0x00002fd0       0x8c obj/uc_libc_dev/sound/beep/beep.o
                0x00002fd0                beep_Tick

.text.cli_GetLine
                0x0000305c       0xf4
 .text.cli_GetLine
                0x0000305c       0xf4 obj/uc_libc_dev/cli/cli.o
                0x0000305c                cli_GetLine

.text.cli_Help  0x00003150       0x98
 .text.cli_Help
                0x00003150       0x98 obj/uc_libc_dev/cli/cli.o
                0x00003150                cli_Help

.text.cli_ArgsParse
                0x000031e8       0xf0
 .text.cli_ArgsParse
                0x000031e8       0xf0 obj/uc_libc_dev/cli/cli.o
                0x000031e8                cli_ArgsParse

.text.cli_ArgsDispatch
                0x000032d8       0xa0
 .text.cli_ArgsDispatch
                0x000032d8       0xa0 obj/uc_libc_dev/cli/cli.o
                0x000032d8                cli_ArgsDispatch

.text.lcd_command
                0x00003378       0x1a
 .text.lcd_command
                0x00003378       0x1a obj/uc_libc_dev/display/liquid_crystal.o

.text.lcd_PutChar
                0x00003392       0x1a
 .text.lcd_PutChar
                0x00003392       0x1a obj/uc_libc_dev/display/liquid_crystal.o
                0x00003392                lcd_PutChar

.text.lcd_Clear
                0x000033ac       0x18
 .text.lcd_Clear
                0x000033ac       0x18 obj/uc_libc_dev/display/liquid_crystal.o
                0x000033ac                lcd_Clear

.text.lcd_SetCursor
                0x000033c4       0x2c
 .text.lcd_SetCursor
                0x000033c4       0x2c obj/uc_libc_dev/display/liquid_crystal.o
                0x000033c4                lcd_SetCursor

.text.lcd_Display
                0x000033f0       0x18
 .text.lcd_Display
                0x000033f0       0x18 obj/uc_libc_dev/display/liquid_crystal.o
                0x000033f0                lcd_Display

.text.lcd_Init  0x00003408       0xb0
 .text.lcd_Init
                0x00003408       0xb0 obj/uc_libc_dev/display/liquid_crystal.o
                0x00003408                lcd_Init

.text.lcd_CreateChar
                0x000034b8       0x3a
 .text.lcd_CreateChar
                0x000034b8       0x3a obj/uc_libc_dev/display/liquid_crystal.o
                0x000034b8                lcd_CreateChar

.text.lcd_printfInit
                0x000034f4       0x20
 .text.lcd_printfInit
                0x000034f4       0x20 obj/uc_libc_dev/display/liquid_crystal.o
                0x000034f4                lcd_printfInit

.text.lcd_printf
                0x00003514       0x5c
 .text.lcd_printf
                0x00003514       0x5c obj/uc_libc_dev/display/liquid_crystal.o
                0x00003514                lcd_printf

.text.lcd_config_ports
                0x00003570       0x28
 .text.lcd_config_ports
                0x00003570       0x28 obj/uc_libc_dev/display/portable/arm_lpc/lcd_drv.o
                0x00003570                lcd_config_ports

.text.lcd_read  0x00003598       0x90
 .text.lcd_read
                0x00003598       0x90 obj/uc_libc_dev/display/portable/arm_lpc/lcd_drv.o
                0x00003598                lcd_read

.text.lcd_write
                0x00003628       0xc8
 .text.lcd_write
                0x00003628       0xc8 obj/uc_libc_dev/display/portable/arm_lpc/lcd_drv.o
                0x00003628                lcd_write

.text.__get_current_locale
                0x000036f0       0x18
 .text.__get_current_locale
                0x000036f0       0x18 d:/cc/arm-yagarto-5.4.2016q3/bin/../lib/gcc/arm-none-eabi/5.4.1/../../../../arm-none-eabi/lib/armv7-m\libc.a(lib_a-locale.o)

.text.__locale_ctype_ptr
                0x00003708       0x14
 .text.__locale_ctype_ptr
                0x00003708       0x14 d:/cc/arm-yagarto-5.4.2016q3/bin/../lib/gcc/arm-none-eabi/5.4.1/../../../../arm-none-eabi/lib/armv7-m\libc.a(lib_a-locale.o)
                0x00003708                __locale_ctype_ptr

.text.__ascii_mbtowc
                0x0000371c       0x2c
 .text.__ascii_mbtowc
                0x0000371c       0x2c d:/cc/arm-yagarto-5.4.2016q3/bin/../lib/gcc/arm-none-eabi/5.4.1/../../../../arm-none-eabi/lib/armv7-m\libc.a(lib_a-mbtowc_r.o)
                0x0000371c                __ascii_mbtowc

.text.memset    0x00003748       0x9c
 .text.memset   0x00003748       0x9c d:/cc/arm-yagarto-5.4.2016q3/bin/../lib/gcc/arm-none-eabi/5.4.1/../../../../arm-none-eabi/lib/armv7-m\libc.a(lib_a-memset.o)
                0x00003748                memset

.text.strlen    0x000037e4       0x5c
 .text.strlen   0x000037e4       0x5c d:/cc/arm-yagarto-5.4.2016q3/bin/../lib/gcc/arm-none-eabi/5.4.1/../../../../arm-none-eabi/lib/armv7-m\libc.a(lib_a-strlen-stub.o)
                0x000037e4                strlen

.text.__ascii_wctomb
                0x00003840       0x1c
 .text.__ascii_wctomb
                0x00003840       0x1c d:/cc/arm-yagarto-5.4.2016q3/bin/../lib/gcc/arm-none-eabi/5.4.1/../../../../arm-none-eabi/lib/armv7-m\libc.a(lib_a-wctomb_r.o)
                0x00003840                __ascii_wctomb
                0x0000385c                . = ALIGN (0x4)

.rodata         0x0000385c      0x88d
 *(.rodata)
 .rodata        0x0000385c       0x2c obj/uc_libc_dev/stdio/stdio_uc.o
 *(.rodata*)
 .rodata.str1.1
                0x00003888      0x356 obj/uc_libc_dev/_arch/arm_lpc/common/vic_cortexm3.o
 .rodata.str1.1
                0x00003bde       0x40 obj/main.o
                                 0x56 (size before relaxing)
 .rodata.str1.1
                0x00003c1e       0x7a obj/app.o
 .rodata.cli_list
                0x00003c98       0x8c obj/prompt.o
 .rodata.str1.1
                0x00003d24      0x1ef obj/prompt.o
                                0x1fa (size before relaxing)
 .rodata.str1.1
                0x00003f13       0x2a obj/uc_libc_dev/misc/utils.o
                                 0x2c (size before relaxing)
 .rodata.str1.1
                0x00003f3d       0x94 obj/uc_libc_dev/cli/cli.o
                                 0x9d (size before relaxing)
 .rodata.str1.1
                0x00003fd1        0x3 obj/uc_libc_dev/display/liquid_crystal.o
 *fill*         0x00003fd1        0x3 
 .rodata.str1.4
                0x00003fd4       0x14 d:/cc/arm-yagarto-5.4.2016q3/bin/../lib/gcc/arm-none-eabi/5.4.1/../../../../arm-none-eabi/lib/armv7-m\libc.a(lib_a-locale.o)
                                 0x12 (size before relaxing)
 .rodata._ctype_
                0x00003fe8      0x101 d:/cc/arm-yagarto-5.4.2016q3/bin/../lib/gcc/arm-none-eabi/5.4.1/../../../../arm-none-eabi/lib/armv7-m\libc.a(lib_a-ctype_.o)
                0x00003fe8                _ctype_

.rel.dyn        0x000040ec        0x0
 .rel.iplt      0x000040ec        0x0 obj/uc_libc_dev/_arch/arm_lpc/common/arm.o
                0x000040ec                . = ALIGN (0x4)
                0x000040ec                _etext = .

.data           0x10000000      0x5d4 load address 0x000040ec
                0x10000000                _data = .
 *(.data)
 *(.data.*)
 .data.heart    0x10000000        0x8 obj/app.o
                0x10000000                heart
 .data.frownie  0x10000008        0x8 obj/app.o
                0x10000008                frownie
 .data.ledpos.4855
                0x10000010        0x4 obj/app.o
 .data.sun      0x10000014        0x8 obj/app.o
                0x10000014                sun
 .data.armsUp   0x1000001c        0x8 obj/app.o
                0x1000001c                armsUp
 .data.smiley   0x10000024        0x8 obj/app.o
                0x10000024                smiley
 .data.armsDown
                0x1000002c        0x8 obj/app.o
                0x1000002c                armsDown
 .data.initGet  0x10000034        0x1 obj/uc_libc_dev/cli/cli.o
 *fill*         0x10000035        0x3 
 .data.__global_locale
                0x10000038      0x16c d:/cc/arm-yagarto-5.4.2016q3/bin/../lib/gcc/arm-none-eabi/5.4.1/../../../../arm-none-eabi/lib/armv7-m\libc.a(lib_a-locale.o)
                0x10000038                __global_locale
 *fill*         0x100001a4        0x4 
 .data.impure_data
                0x100001a8      0x428 d:/cc/arm-yagarto-5.4.2016q3/bin/../lib/gcc/arm-none-eabi/5.4.1/../../../../arm-none-eabi/lib/armv7-m\libc.a(lib_a-impure.o)
 .data._impure_ptr
                0x100005d0        0x4 d:/cc/arm-yagarto-5.4.2016q3/bin/../lib/gcc/arm-none-eabi/5.4.1/../../../../arm-none-eabi/lib/armv7-m\libc.a(lib_a-impure.o)
                0x100005d0                _impure_ptr

.igot.plt       0x100005d4        0x0 load address 0x000046c0
 .igot.plt      0x100005d4        0x0 obj/uc_libc_dev/_arch/arm_lpc/common/arm.o
                0x100005d4                . = ALIGN (0x4)
                0x100005d4                _edata = .

.bss            0x100005d4       0x25 load address 0x000046c0
                0x100005d4                _bss = .
 *(.bss)
 *(COMMON)
 COMMON         0x100005d4       0x18 obj/main.o
                0x100005d4                control
 COMMON         0x100005ec        0x4 obj/uc_libc_dev/keyboard/gkey.o
                0x100005ec                gkey_FastInc
 COMMON         0x100005f0        0x9 obj/uc_libc_dev/display/liquid_crystal.o
                0x100005f0                _row_offsets
                0x100005f4                _displaycontrol
                0x100005f5                _numlines
                0x100005f6                _displaymode
                0x100005f7                _displayfunction
                0x100005f8                _cols

.bss.vicerr_Functions
                0x100005fc        0x4 load address 0x000046e8
 .bss.vicerr_Functions
                0x100005fc        0x4 obj/uc_libc_dev/_arch/arm_lpc/common/vic_cortexm3.o

.bss.countTicksLed
                0x10000600        0x4 load address 0x000046ec
 .bss.countTicksLed
                0x10000600        0x4 obj/uc_libc_dev/_arch/arm_lpc/timer/systick.o

.bss.countTicks_ms
                0x10000604        0x4 load address 0x000046f0
 .bss.countTicks_ms
                0x10000604        0x4 obj/uc_libc_dev/_arch/arm_lpc/timer/systick.o

.bss.callfuncTime
                0x10000608        0x4 load address 0x000046f4
 .bss.callfuncTime
                0x10000608        0x4 obj/uc_libc_dev/_arch/arm_lpc/timer/systick.o

.bss.systime_IntFunctions
                0x1000060c        0x4 load address 0x000046f8
 .bss.systime_IntFunctions
                0x1000060c        0x4 obj/uc_libc_dev/_arch/arm_lpc/timer/systick.o

.bss.u0_data_tx
                0x10000610       0x96 load address 0x000046fc
 .bss.u0_data_tx
                0x10000610       0x96 obj/uc_libc_dev/_arch/arm_lpc/uart/uart0_irq.o

.bss.u0_tx_running
                0x100006a6        0x1 load address 0x00004792
 .bss.u0_tx_running
                0x100006a6        0x1 obj/uc_libc_dev/_arch/arm_lpc/uart/uart0_irq.o

.bss.u0_overflow_rx
                0x100006a8        0x2 load address 0x00004794
 .bss.u0_overflow_rx
                0x100006a8        0x2 obj/uc_libc_dev/_arch/arm_lpc/uart/uart0_irq.o

.bss.u0_buf_rx  0x100006ac        0xc load address 0x00004798
 .bss.u0_buf_rx
                0x100006ac        0xc obj/uc_libc_dev/_arch/arm_lpc/uart/uart0_irq.o

.bss.u0_buf_tx  0x100006b8        0xc load address 0x000047a4
 .bss.u0_buf_tx
                0x100006b8        0xc obj/uc_libc_dev/_arch/arm_lpc/uart/uart0_irq.o

.bss.u0_data_rx
                0x100006c4       0x96 load address 0x000047b0
 .bss.u0_data_rx
                0x100006c4       0x96 obj/uc_libc_dev/_arch/arm_lpc/uart/uart0_irq.o

.bss.x.4895     0x1000075c        0x4 load address 0x00004848
 .bss.x.4895    0x1000075c        0x4 obj/main.o

.bss.ticks_d.4856
                0x10000760        0x4 load address 0x0000484c
 .bss.ticks_d.4856
                0x10000760        0x4 obj/app.o

.bss.bufKey.4850
                0x10000764        0xc load address 0x00004850
 .bss.bufKey.4850
                0x10000764        0xc obj/app.o

.bss.timeReadKey.4849
                0x10000770        0x4 load address 0x0000485c
 .bss.timeReadKey.4849
                0x10000770        0x4 obj/app.o

.bss.idx.4851   0x10000774        0x4 load address 0x00004860
 .bss.idx.4851  0x10000774        0x4 obj/app.o

.bss.argc_prompt
                0x10000778        0x4 load address 0x00004864
 .bss.argc_prompt
                0x10000778        0x4 obj/prompt.o

.bss.result_prompt
                0x1000077c        0x4 load address 0x00004868
 .bss.result_prompt
                0x1000077c        0x4 obj/prompt.o

.bss.argv_prompt
                0x10000780       0x28 load address 0x0000486c
 .bss.argv_prompt
                0x10000780       0x28 obj/prompt.o

.bss.buffer_prompt
                0x100007a8       0x28 load address 0x00004894
 .bss.buffer_prompt
                0x100007a8       0x28 obj/prompt.o

.bss.dev1_putc  0x100007d0        0x4 load address 0x000048bc
 .bss.dev1_putc
                0x100007d0        0x4 obj/uc_libc_dev/stdio/stdio_uc.o

.bss.dev2_putc  0x100007d4        0x4 load address 0x000048c0
 .bss.dev2_putc
                0x100007d4        0x4 obj/uc_libc_dev/stdio/stdio_uc.o

.bss.stdio_putc
                0x100007d8        0x4 load address 0x000048c4
 .bss.stdio_putc
                0x100007d8        0x4 obj/uc_libc_dev/stdio/stdio_uc.o

.bss.dev4_putc  0x100007dc        0x4 load address 0x000048c8
 .bss.dev4_putc
                0x100007dc        0x4 obj/uc_libc_dev/stdio/stdio_uc.o

.bss.dev3_putc  0x100007e0        0x4 load address 0x000048cc
 .bss.dev3_putc
                0x100007e0        0x4 obj/uc_libc_dev/stdio/stdio_uc.o

.bss.putcharfunc.4764
                0x100007e4        0x4 load address 0x000048d0
 .bss.putcharfunc.4764
                0x100007e4        0x4 obj/uc_libc_dev/stdio/stdio_uc.o

.bss.stdio_getc
                0x100007e8        0x4 load address 0x000048d4
 .bss.stdio_getc
                0x100007e8        0x4 obj/uc_libc_dev/stdio/stdio_uc.o

.bss.debug_putc
                0x100007ec        0x4 load address 0x000048d8
 .bss.debug_putc
                0x100007ec        0x4 obj/uc_libc_dev/stdio/stdio_uc.o

.bss.err_putc   0x100007f0        0x4 load address 0x000048dc
 .bss.err_putc  0x100007f0        0x4 obj/uc_libc_dev/stdio/stdio_uc.o

.bss.nTimes.4279
                0x100007f4        0x4 load address 0x000048e0
 .bss.nTimes.4279
                0x100007f4        0x4 obj/uc_libc_dev/misc/led_error.o

.bss.ff.4278    0x100007f8        0x4 load address 0x000048e4
 .bss.ff.4278   0x100007f8        0x4 obj/uc_libc_dev/misc/led_error.o

.bss.count2.4277
                0x100007fc        0x4 load address 0x000048e8
 .bss.count2.4277
                0x100007fc        0x4 obj/uc_libc_dev/misc/led_error.o

.bss.error      0x10000800        0x4 load address 0x000048ec
 .bss.error     0x10000800        0x4 obj/uc_libc_dev/misc/led_error.o

.bss.ledBlink   0x10000804        0x4 load address 0x000048f0
 .bss.ledBlink  0x10000804        0x4 obj/uc_libc_dev/misc/led_error.o

.bss.count1.4276
                0x10000808        0x4 load address 0x000048f4
 .bss.count1.4276
                0x10000808        0x4 obj/uc_libc_dev/misc/led_error.o

.bss.onKeyUp    0x1000080c        0x4 load address 0x000048f8
 .bss.onKeyUp   0x1000080c        0x4 obj/uc_libc_dev/keyboard/gkey.o

.bss.timeRepeat
                0x10000810        0x4 load address 0x000048fc
 .bss.timeRepeat
                0x10000810        0x4 obj/uc_libc_dev/keyboard/gkey.o

.bss.estado.4276
                0x10000814        0x1 load address 0x00004900
 .bss.estado.4276
                0x10000814        0x1 obj/uc_libc_dev/keyboard/gkey.o

.bss.onKeyDown  0x10000818        0x4 load address 0x00004904
 .bss.onKeyDown
                0x10000818        0x4 obj/uc_libc_dev/keyboard/gkey.o

.bss.keynow.4275
                0x1000081c        0x1 load address 0x00004908
 .bss.keynow.4275
                0x1000081c        0x1 obj/uc_libc_dev/keyboard/gkey.o

.bss.repeat.4277
                0x10000820        0x4 load address 0x0000490c
 .bss.repeat.4277
                0x10000820        0x4 obj/uc_libc_dev/keyboard/gkey.o

.bss.onKeyPress
                0x10000824        0x4 load address 0x00004910
 .bss.onKeyPress
                0x10000824        0x4 obj/uc_libc_dev/keyboard/gkey.o

.bss.beep       0x10000828       0x30 load address 0x00004914
 .bss.beep      0x10000828       0x30 obj/uc_libc_dev/sound/beep/beep.o

.bss.cmd_list_active
                0x10000858        0x4 load address 0x00004944
 .bss.cmd_list_active
                0x10000858        0x4 obj/uc_libc_dev/cli/cli.o
                0x10000858                cmd_list_active

.bss.p          0x1000085c        0x4 load address 0x00004948
 .bss.p         0x1000085c        0x4 obj/uc_libc_dev/cli/cli.o

.bss.c          0x10000860        0x1 load address 0x0000494c
 .bss.c         0x10000860        0x1 obj/uc_libc_dev/cli/cli.o

.bss.devicePrintf
                0x10000864        0x4 load address 0x00004950
 .bss.devicePrintf
                0x10000864        0x4 obj/uc_libc_dev/display/liquid_crystal.o
                0x10000868                . = ALIGN (0x4)
                0x10000868                _ebss = .
                0x10000868                _end = .
                [!provide]                PROVIDE (end, .)

.stab
 *(.stab)

.stabstr
 *(.stabstr)

.stab.excl
 *(.stab.excl)

.stab.exclstr
 *(.stab.exclstr)

.stab.index
 *(.stab.index)

.stab.indexstr
 *(.stab.indexstr)

.comment        0x00000000       0x6e
 *(.comment)
 .comment       0x00000000       0x6e obj/uc_libc_dev/_arch/arm_lpc/common/arm.o
                                 0x6f (size before relaxing)
 .comment       0x0000006e       0x6f obj/uc_libc_dev/_arch/arm_lpc/common/startup/startup.o
 .comment       0x0000006e       0x6f obj/uc_libc_dev/_arch/arm_lpc/common/vic_cortexm3.o
 .comment       0x0000006e       0x6f obj/uc_libc_dev/_arch/arm_lpc/timer/systick.o
 .comment       0x0000006e       0x6f obj/uc_libc_dev/_arch/arm_lpc/timer/delay.o
 .comment       0x0000006e       0x6f obj/uc_libc_dev/_arch/arm_lpc/uart/uart0_irq.o
 .comment       0x0000006e       0x6f obj/main.o
 .comment       0x0000006e       0x6f obj/app.o
 .comment       0x0000006e       0x6f obj/prompt.o
 .comment       0x0000006e       0x6f obj/uc_libc_dev/stdio/stdio_uc.o
 .comment       0x0000006e       0x6f obj/uc_libc_dev/misc/buffer.o
 .comment       0x0000006e       0x6f obj/uc_libc_dev/misc/utils.o
 .comment       0x0000006e       0x6f obj/uc_libc_dev/misc/led_error.o
 .comment       0x0000006e       0x6f obj/uc_libc_dev/keyboard/gkey.o
 .comment       0x0000006e       0x6f obj/uc_libc_dev/sound/beep/beep.o
 .comment       0x0000006e       0x6f obj/uc_libc_dev/cli/cli.o
 .comment       0x0000006e       0x6f obj/uc_libc_dev/display/liquid_crystal.o
 .comment       0x0000006e       0x6f obj/uc_libc_dev/display/portable/arm_lpc/lcd_drv.o

.ARM.attributes
                0x00000000       0x31
 .ARM.attributes
                0x00000000       0x33 obj/uc_libc_dev/_arch/arm_lpc/common/arm.o
 .ARM.attributes
                0x00000033       0x33 obj/uc_libc_dev/_arch/arm_lpc/common/startup/startup.o
 .ARM.attributes
                0x00000066       0x33 obj/uc_libc_dev/_arch/arm_lpc/common/vic_cortexm3.o
 .ARM.attributes
                0x00000099       0x33 obj/uc_libc_dev/_arch/arm_lpc/timer/systick.o
 .ARM.attributes
                0x000000cc       0x33 obj/uc_libc_dev/_arch/arm_lpc/timer/delay.o
 .ARM.attributes
                0x000000ff       0x33 obj/uc_libc_dev/_arch/arm_lpc/uart/uart0_irq.o
 .ARM.attributes
                0x00000132       0x33 obj/main.o
 .ARM.attributes
                0x00000165       0x33 obj/app.o
 .ARM.attributes
                0x00000198       0x33 obj/prompt.o
 .ARM.attributes
                0x000001cb       0x33 obj/uc_libc_dev/stdio/stdio_uc.o
 .ARM.attributes
                0x000001fe       0x33 obj/uc_libc_dev/misc/buffer.o
 .ARM.attributes
                0x00000231       0x33 obj/uc_libc_dev/misc/utils.o
 .ARM.attributes
                0x00000264       0x33 obj/uc_libc_dev/misc/led_error.o
 .ARM.attributes
                0x00000297       0x33 obj/uc_libc_dev/keyboard/gkey.o
 .ARM.attributes
                0x000002ca       0x33 obj/uc_libc_dev/sound/beep/beep.o
 .ARM.attributes
                0x000002fd       0x33 obj/uc_libc_dev/cli/cli.o
 .ARM.attributes
                0x00000330       0x33 obj/uc_libc_dev/display/liquid_crystal.o
 .ARM.attributes
                0x00000363       0x33 obj/uc_libc_dev/display/portable/arm_lpc/lcd_drv.o
 .ARM.attributes
                0x00000396       0x1d d:/cc/arm-yagarto-5.4.2016q3/bin/../lib/gcc/arm-none-eabi/5.4.1/armv7-m\libgcc.a(_arm_addsubdf3.o)
 .ARM.attributes
                0x000003b3       0x1d d:/cc/arm-yagarto-5.4.2016q3/bin/../lib/gcc/arm-none-eabi/5.4.1/armv7-m\libgcc.a(_arm_muldivdf3.o)
 .ARM.attributes
                0x000003d0       0x1d d:/cc/arm-yagarto-5.4.2016q3/bin/../lib/gcc/arm-none-eabi/5.4.1/armv7-m\libgcc.a(_arm_cmpdf2.o)
 .ARM.attributes
                0x000003ed       0x1d d:/cc/arm-yagarto-5.4.2016q3/bin/../lib/gcc/arm-none-eabi/5.4.1/armv7-m\libgcc.a(_arm_fixdfsi.o)
 .ARM.attributes
                0x0000040a       0x1d d:/cc/arm-yagarto-5.4.2016q3/bin/../lib/gcc/arm-none-eabi/5.4.1/armv7-m\libgcc.a(_arm_addsubsf3.o)
 .ARM.attributes
                0x00000427       0x1d d:/cc/arm-yagarto-5.4.2016q3/bin/../lib/gcc/arm-none-eabi/5.4.1/armv7-m\libgcc.a(_arm_muldivsf3.o)
 .ARM.attributes
                0x00000444       0x2d d:/cc/arm-yagarto-5.4.2016q3/bin/../lib/gcc/arm-none-eabi/5.4.1/../../../../arm-none-eabi/lib/armv7-m\libc.a(lib_a-locale.o)
 .ARM.attributes
                0x00000471       0x2d d:/cc/arm-yagarto-5.4.2016q3/bin/../lib/gcc/arm-none-eabi/5.4.1/../../../../arm-none-eabi/lib/armv7-m\libc.a(lib_a-mbtowc_r.o)
 .ARM.attributes
                0x0000049e       0x2d d:/cc/arm-yagarto-5.4.2016q3/bin/../lib/gcc/arm-none-eabi/5.4.1/../../../../arm-none-eabi/lib/armv7-m\libc.a(lib_a-memset.o)
 .ARM.attributes
                0x000004cb       0x1b d:/cc/arm-yagarto-5.4.2016q3/bin/../lib/gcc/arm-none-eabi/5.4.1/../../../../arm-none-eabi/lib/armv7-m\libc.a(lib_a-strcmp.o)
 .ARM.attributes
                0x000004e6       0x2d d:/cc/arm-yagarto-5.4.2016q3/bin/../lib/gcc/arm-none-eabi/5.4.1/../../../../arm-none-eabi/lib/armv7-m\libc.a(lib_a-strlen-stub.o)
 .ARM.attributes
                0x00000513       0x2d d:/cc/arm-yagarto-5.4.2016q3/bin/../lib/gcc/arm-none-eabi/5.4.1/../../../../arm-none-eabi/lib/armv7-m\libc.a(lib_a-wctomb_r.o)
 .ARM.attributes
                0x00000540       0x2d d:/cc/arm-yagarto-5.4.2016q3/bin/../lib/gcc/arm-none-eabi/5.4.1/../../../../arm-none-eabi/lib/armv7-m\libc.a(lib_a-ctype_.o)
 .ARM.attributes
                0x0000056d       0x2d d:/cc/arm-yagarto-5.4.2016q3/bin/../lib/gcc/arm-none-eabi/5.4.1/../../../../arm-none-eabi/lib/armv7-m\libc.a(lib_a-impure.o)

.debug
 *(.debug)

.line
 *(.line)

.debug_srcinfo
 *(.debug_srcinfo)

.debug_sfnames
 *(.debug_sfnames)

.debug_aranges  0x00000000      0x738
 *(.debug_aranges)
 .debug_aranges
                0x00000000       0x28 obj/uc_libc_dev/_arch/arm_lpc/common/arm.o
 .debug_aranges
                0x00000028       0x20 obj/uc_libc_dev/_arch/arm_lpc/common/startup/startup.o
 .debug_aranges
                0x00000048      0x1e0 obj/uc_libc_dev/_arch/arm_lpc/common/vic_cortexm3.o
 .debug_aranges
                0x00000228       0x60 obj/uc_libc_dev/_arch/arm_lpc/timer/systick.o
 .debug_aranges
                0x00000288       0x20 obj/uc_libc_dev/_arch/arm_lpc/timer/delay.o
 .debug_aranges
                0x000002a8       0x98 obj/uc_libc_dev/_arch/arm_lpc/uart/uart0_irq.o
 .debug_aranges
                0x00000340       0x28 obj/main.o
 .debug_aranges
                0x00000368       0x60 obj/app.o
 .debug_aranges
                0x000003c8       0x48 obj/prompt.o
 .debug_aranges
                0x00000410       0xa8 obj/uc_libc_dev/stdio/stdio_uc.o
 .debug_aranges
                0x000004b8       0x58 obj/uc_libc_dev/misc/buffer.o
 .debug_aranges
                0x00000510       0x58 obj/uc_libc_dev/misc/utils.o
 .debug_aranges
                0x00000568       0x30 obj/uc_libc_dev/misc/led_error.o
 .debug_aranges
                0x00000598       0x30 obj/uc_libc_dev/keyboard/gkey.o
 .debug_aranges
                0x000005c8       0x48 obj/uc_libc_dev/sound/beep/beep.o
 .debug_aranges
                0x00000610       0x38 obj/uc_libc_dev/cli/cli.o
 .debug_aranges
                0x00000648       0xc0 obj/uc_libc_dev/display/liquid_crystal.o
 .debug_aranges
                0x00000708       0x30 obj/uc_libc_dev/display/portable/arm_lpc/lcd_drv.o

.debug_pubnames
 *(.debug_pubnames)

.debug_info     0x00000000     0x5e51
 *(.debug_info .gnu.linkonce.wi.*)
 .debug_info    0x00000000       0xe6 obj/uc_libc_dev/_arch/arm_lpc/common/arm.o
 .debug_info    0x000000e6      0x132 obj/uc_libc_dev/_arch/arm_lpc/common/startup/startup.o
 .debug_info    0x00000218     0x10bd obj/uc_libc_dev/_arch/arm_lpc/common/vic_cortexm3.o
 .debug_info    0x000012d5      0x30e obj/uc_libc_dev/_arch/arm_lpc/timer/systick.o
 .debug_info    0x000015e3       0xac obj/uc_libc_dev/_arch/arm_lpc/timer/delay.o
 .debug_info    0x0000168f      0x73b obj/uc_libc_dev/_arch/arm_lpc/uart/uart0_irq.o
 .debug_info    0x00001dca      0x409 obj/main.o
 .debug_info    0x000021d3      0x6b1 obj/app.o
 .debug_info    0x00002884      0x7da obj/prompt.o
 .debug_info    0x0000305e      0xec4 obj/uc_libc_dev/stdio/stdio_uc.o
 .debug_info    0x00003f22      0x29e obj/uc_libc_dev/misc/buffer.o
 .debug_info    0x000041c0      0x58e obj/uc_libc_dev/misc/utils.o
 .debug_info    0x0000474e      0x1fd obj/uc_libc_dev/misc/led_error.o
 .debug_info    0x0000494b      0x1dd obj/uc_libc_dev/keyboard/gkey.o
 .debug_info    0x00004b28      0x223 obj/uc_libc_dev/sound/beep/beep.o
 .debug_info    0x00004d4b      0x673 obj/uc_libc_dev/cli/cli.o
 .debug_info    0x000053be      0x926 obj/uc_libc_dev/display/liquid_crystal.o
 .debug_info    0x00005ce4      0x16d obj/uc_libc_dev/display/portable/arm_lpc/lcd_drv.o

.debug_abbrev   0x00000000     0x1d5a
 *(.debug_abbrev)
 .debug_abbrev  0x00000000       0xa2 obj/uc_libc_dev/_arch/arm_lpc/common/arm.o
 .debug_abbrev  0x000000a2       0xa9 obj/uc_libc_dev/_arch/arm_lpc/common/startup/startup.o
 .debug_abbrev  0x0000014b      0x196 obj/uc_libc_dev/_arch/arm_lpc/common/vic_cortexm3.o
 .debug_abbrev  0x000002e1      0x165 obj/uc_libc_dev/_arch/arm_lpc/timer/systick.o
 .debug_abbrev  0x00000446       0x60 obj/uc_libc_dev/_arch/arm_lpc/timer/delay.o
 .debug_abbrev  0x000004a6      0x331 obj/uc_libc_dev/_arch/arm_lpc/uart/uart0_irq.o
 .debug_abbrev  0x000007d7      0x122 obj/main.o
 .debug_abbrev  0x000008f9      0x1f2 obj/app.o
 .debug_abbrev  0x00000aeb      0x2a3 obj/prompt.o
 .debug_abbrev  0x00000d8e      0x387 obj/uc_libc_dev/stdio/stdio_uc.o
 .debug_abbrev  0x00001115      0x125 obj/uc_libc_dev/misc/buffer.o
 .debug_abbrev  0x0000123a      0x1a2 obj/uc_libc_dev/misc/utils.o
 .debug_abbrev  0x000013dc      0x12d obj/uc_libc_dev/misc/led_error.o
 .debug_abbrev  0x00001509      0x11f obj/uc_libc_dev/keyboard/gkey.o
 .debug_abbrev  0x00001628      0x12e obj/uc_libc_dev/sound/beep/beep.o
 .debug_abbrev  0x00001756      0x242 obj/uc_libc_dev/cli/cli.o
 .debug_abbrev  0x00001998      0x2c4 obj/uc_libc_dev/display/liquid_crystal.o
 .debug_abbrev  0x00001c5c       0xfe obj/uc_libc_dev/display/portable/arm_lpc/lcd_drv.o

.debug_line     0x00000000     0x221f
 *(.debug_line)
 .debug_line    0x00000000       0xd0 obj/uc_libc_dev/_arch/arm_lpc/common/arm.o
 .debug_line    0x000000d0       0x93 obj/uc_libc_dev/_arch/arm_lpc/common/startup/startup.o
 .debug_line    0x00000163      0x5d0 obj/uc_libc_dev/_arch/arm_lpc/common/vic_cortexm3.o
 .debug_line    0x00000733      0x14f obj/uc_libc_dev/_arch/arm_lpc/timer/systick.o
 .debug_line    0x00000882       0x7c obj/uc_libc_dev/_arch/arm_lpc/timer/delay.o
 .debug_line    0x000008fe      0x2a4 obj/uc_libc_dev/_arch/arm_lpc/uart/uart0_irq.o
 .debug_line    0x00000ba2      0x1f1 obj/main.o
 .debug_line    0x00000d93      0x306 obj/app.o
 .debug_line    0x00001099      0x1b6 obj/prompt.o
 .debug_line    0x0000124f      0x383 obj/uc_libc_dev/stdio/stdio_uc.o
 .debug_line    0x000015d2      0x10a obj/uc_libc_dev/misc/buffer.o
 .debug_line    0x000016dc      0x231 obj/uc_libc_dev/misc/utils.o
 .debug_line    0x0000190d       0xc6 obj/uc_libc_dev/misc/led_error.o
 .debug_line    0x000019d3       0xf1 obj/uc_libc_dev/keyboard/gkey.o
 .debug_line    0x00001ac4      0x10a obj/uc_libc_dev/sound/beep/beep.o
 .debug_line    0x00001bce      0x1ca obj/uc_libc_dev/cli/cli.o
 .debug_line    0x00001d98      0x360 obj/uc_libc_dev/display/liquid_crystal.o
 .debug_line    0x000020f8      0x127 obj/uc_libc_dev/display/portable/arm_lpc/lcd_drv.o

.debug_frame    0x00000000     0x156c
 *(.debug_frame)
 .debug_frame   0x00000000       0x40 obj/uc_libc_dev/_arch/arm_lpc/common/arm.o
 .debug_frame   0x00000040       0x2c obj/uc_libc_dev/_arch/arm_lpc/common/startup/startup.o
 .debug_frame   0x0000006c      0x608 obj/uc_libc_dev/_arch/arm_lpc/common/vic_cortexm3.o
 .debug_frame   0x00000674       0xac obj/uc_libc_dev/_arch/arm_lpc/timer/systick.o
 .debug_frame   0x00000720       0x20 obj/uc_libc_dev/_arch/arm_lpc/timer/delay.o
 .debug_frame   0x00000740      0x1c0 obj/uc_libc_dev/_arch/arm_lpc/uart/uart0_irq.o
 .debug_frame   0x00000900       0x4c obj/main.o
 .debug_frame   0x0000094c      0x104 obj/app.o
 .debug_frame   0x00000a50       0xd8 obj/prompt.o
 .debug_frame   0x00000b28      0x248 obj/uc_libc_dev/stdio/stdio_uc.o
 .debug_frame   0x00000d70       0xc0 obj/uc_libc_dev/misc/buffer.o
 .debug_frame   0x00000e30      0x13c obj/uc_libc_dev/misc/utils.o
 .debug_frame   0x00000f6c       0x50 obj/uc_libc_dev/misc/led_error.o
 .debug_frame   0x00000fbc       0x50 obj/uc_libc_dev/keyboard/gkey.o
 .debug_frame   0x0000100c       0x88 obj/uc_libc_dev/sound/beep/beep.o
 .debug_frame   0x00001094       0xd8 obj/uc_libc_dev/cli/cli.o
 .debug_frame   0x0000116c      0x210 obj/uc_libc_dev/display/liquid_crystal.o
 .debug_frame   0x0000137c       0x5c obj/uc_libc_dev/display/portable/arm_lpc/lcd_drv.o
 .debug_frame   0x000013d8       0x84 d:/cc/arm-yagarto-5.4.2016q3/bin/../lib/gcc/arm-none-eabi/5.4.1/../../../../arm-none-eabi/lib/armv7-m\libc.a(lib_a-locale.o)
 .debug_frame   0x0000145c       0x4c d:/cc/arm-yagarto-5.4.2016q3/bin/../lib/gcc/arm-none-eabi/5.4.1/../../../../arm-none-eabi/lib/armv7-m\libc.a(lib_a-mbtowc_r.o)
 .debug_frame   0x000014a8       0x34 d:/cc/arm-yagarto-5.4.2016q3/bin/../lib/gcc/arm-none-eabi/5.4.1/../../../../arm-none-eabi/lib/armv7-m\libc.a(lib_a-memset.o)
 .debug_frame   0x000014dc       0x34 d:/cc/arm-yagarto-5.4.2016q3/bin/../lib/gcc/arm-none-eabi/5.4.1/../../../../arm-none-eabi/lib/armv7-m\libc.a(lib_a-strcmp.o)
 .debug_frame   0x00001510       0x20 d:/cc/arm-yagarto-5.4.2016q3/bin/../lib/gcc/arm-none-eabi/5.4.1/../../../../arm-none-eabi/lib/armv7-m\libc.a(lib_a-strlen-stub.o)
 .debug_frame   0x00001530       0x3c d:/cc/arm-yagarto-5.4.2016q3/bin/../lib/gcc/arm-none-eabi/5.4.1/../../../../arm-none-eabi/lib/armv7-m\libc.a(lib_a-wctomb_r.o)

.debug_str      0x00000000     0x132f
 *(.debug_str)
 .debug_str     0x00000000      0x190 obj/uc_libc_dev/_arch/arm_lpc/common/arm.o
                                0x1c9 (size before relaxing)
 .debug_str     0x00000190       0x69 obj/uc_libc_dev/_arch/arm_lpc/common/startup/startup.o
                                0x1f6 (size before relaxing)
 .debug_str     0x000001f9      0x2f0 obj/uc_libc_dev/_arch/arm_lpc/common/vic_cortexm3.o
                                0x487 (size before relaxing)
 .debug_str     0x000004e9      0x14b obj/uc_libc_dev/_arch/arm_lpc/timer/systick.o
                                0x2e6 (size before relaxing)
 .debug_str     0x00000634       0x37 obj/uc_libc_dev/_arch/arm_lpc/timer/delay.o
                                0x1bb (size before relaxing)
 .debug_str     0x0000066b      0x238 obj/uc_libc_dev/_arch/arm_lpc/uart/uart0_irq.o
                                0x3fd (size before relaxing)
 .debug_str     0x000008a3       0xee obj/main.o
                                0x2e7 (size before relaxing)
 .debug_str     0x00000991      0x107 obj/app.o
                                0x2e7 (size before relaxing)
 .debug_str     0x00000a98      0x179 obj/prompt.o
                                0x369 (size before relaxing)
 .debug_str     0x00000c11      0x203 obj/uc_libc_dev/stdio/stdio_uc.o
                                0x411 (size before relaxing)
 .debug_str     0x00000e14       0x5b obj/uc_libc_dev/misc/buffer.o
                                0x277 (size before relaxing)
 .debug_str     0x00000e6f       0x9d obj/uc_libc_dev/misc/utils.o
                                0x246 (size before relaxing)
 .debug_str     0x00000f0c       0x71 obj/uc_libc_dev/misc/led_error.o
                                0x21c (size before relaxing)
 .debug_str     0x00000f7d       0x63 obj/uc_libc_dev/keyboard/gkey.o
                                0x237 (size before relaxing)
 .debug_str     0x00000fe0       0x86 obj/uc_libc_dev/sound/beep/beep.o
                                0x23e (size before relaxing)
 .debug_str     0x00001066       0xc8 obj/uc_libc_dev/cli/cli.o
                                0x341 (size before relaxing)
 .debug_str     0x0000112e      0x1cc obj/uc_libc_dev/display/liquid_crystal.o
                                0x45f (size before relaxing)
 .debug_str     0x000012fa       0x35 obj/uc_libc_dev/display/portable/arm_lpc/lcd_drv.o
                                0x1e9 (size before relaxing)

.debug_loc      0x00000000     0x37a0
 *(.debug_loc)
 .debug_loc     0x00000000       0x20 obj/uc_libc_dev/_arch/arm_lpc/common/arm.o
 .debug_loc     0x00000020       0x6e obj/uc_libc_dev/_arch/arm_lpc/common/startup/startup.o
 .debug_loc     0x0000008e      0x967 obj/uc_libc_dev/_arch/arm_lpc/common/vic_cortexm3.o
 .debug_loc     0x000009f5       0x67 obj/uc_libc_dev/_arch/arm_lpc/timer/systick.o
 .debug_loc     0x00000a5c      0x567 obj/uc_libc_dev/_arch/arm_lpc/uart/uart0_irq.o
 .debug_loc     0x00000fc3       0x61 obj/main.o
 .debug_loc     0x00001024      0x1e8 obj/app.o
 .debug_loc     0x0000120c      0x2eb obj/prompt.o
 .debug_loc     0x000014f7      0xd3c obj/uc_libc_dev/stdio/stdio_uc.o
 .debug_loc     0x00002233      0x1a7 obj/uc_libc_dev/misc/buffer.o
 .debug_loc     0x000023da      0x88c obj/uc_libc_dev/misc/utils.o
 .debug_loc     0x00002c66       0x5c obj/uc_libc_dev/misc/led_error.o
 .debug_loc     0x00002cc2       0xb3 obj/uc_libc_dev/keyboard/gkey.o
 .debug_loc     0x00002d75       0xe2 obj/uc_libc_dev/sound/beep/beep.o
 .debug_loc     0x00002e57      0x47f obj/uc_libc_dev/cli/cli.o
 .debug_loc     0x000032d6      0x3fd obj/uc_libc_dev/display/liquid_crystal.o
 .debug_loc     0x000036d3       0xcd obj/uc_libc_dev/display/portable/arm_lpc/lcd_drv.o

.debug_macinfo
 *(.debug_macinfo)

.debug_weaknames
 *(.debug_weaknames)

.debug_funcnames
 *(.debug_funcnames)

.debug_typenames
 *(.debug_typenames)

.debug_varnames
 *(.debug_varnames)
OUTPUT(bin/main.elf elf32-littlearm)

.debug_ranges   0x00000000      0x758
 .debug_ranges  0x00000000       0x30 obj/uc_libc_dev/_arch/arm_lpc/common/arm.o
 .debug_ranges  0x00000030       0x10 obj/uc_libc_dev/_arch/arm_lpc/common/startup/startup.o
 .debug_ranges  0x00000040      0x1d0 obj/uc_libc_dev/_arch/arm_lpc/common/vic_cortexm3.o
 .debug_ranges  0x00000210       0x50 obj/uc_libc_dev/_arch/arm_lpc/timer/systick.o
 .debug_ranges  0x00000260       0x10 obj/uc_libc_dev/_arch/arm_lpc/timer/delay.o
 .debug_ranges  0x00000270       0xc0 obj/uc_libc_dev/_arch/arm_lpc/uart/uart0_irq.o
 .debug_ranges  0x00000330       0x18 obj/main.o
 .debug_ranges  0x00000348       0x50 obj/app.o
 .debug_ranges  0x00000398       0x50 obj/prompt.o
 .debug_ranges  0x000003e8       0xf8 obj/uc_libc_dev/stdio/stdio_uc.o
 .debug_ranges  0x000004e0       0x48 obj/uc_libc_dev/misc/buffer.o
 .debug_ranges  0x00000528       0x48 obj/uc_libc_dev/misc/utils.o
 .debug_ranges  0x00000570       0x50 obj/uc_libc_dev/misc/led_error.o
 .debug_ranges  0x000005c0       0x20 obj/uc_libc_dev/keyboard/gkey.o
 .debug_ranges  0x000005e0       0x38 obj/uc_libc_dev/sound/beep/beep.o
 .debug_ranges  0x00000618       0x58 obj/uc_libc_dev/cli/cli.o
 .debug_ranges  0x00000670       0xc8 obj/uc_libc_dev/display/liquid_crystal.o
 .debug_ranges  0x00000738       0x20 obj/uc_libc_dev/display/portable/arm_lpc/lcd_drv.o

Cross Reference Table

Symbol                                            File
_PathLocale                                       d:/cc/arm-yagarto-5.4.2016q3/bin/../lib/gcc/arm-none-eabi/5.4.1/../../../../arm-none-eabi/lib/armv7-m\libc.a(lib_a-locale.o)
__adddf3                                          d:/cc/arm-yagarto-5.4.2016q3/bin/../lib/gcc/arm-none-eabi/5.4.1/armv7-m\libgcc.a(_arm_addsubdf3.o)
__addsf3                                          d:/cc/arm-yagarto-5.4.2016q3/bin/../lib/gcc/arm-none-eabi/5.4.1/armv7-m\libgcc.a(_arm_addsubsf3.o)
__aeabi_cdcmpeq                                   d:/cc/arm-yagarto-5.4.2016q3/bin/../lib/gcc/arm-none-eabi/5.4.1/armv7-m\libgcc.a(_arm_cmpdf2.o)
__aeabi_cdcmple                                   d:/cc/arm-yagarto-5.4.2016q3/bin/../lib/gcc/arm-none-eabi/5.4.1/armv7-m\libgcc.a(_arm_cmpdf2.o)
__aeabi_cdrcmple                                  d:/cc/arm-yagarto-5.4.2016q3/bin/../lib/gcc/arm-none-eabi/5.4.1/armv7-m\libgcc.a(_arm_cmpdf2.o)
__aeabi_d2iz                                      d:/cc/arm-yagarto-5.4.2016q3/bin/../lib/gcc/arm-none-eabi/5.4.1/armv7-m\libgcc.a(_arm_fixdfsi.o)
                                                  obj/uc_libc_dev/stdio/stdio_uc.o
                                                  obj/uc_libc_dev/_arch/arm_lpc/uart/uart0_irq.o
__aeabi_dadd                                      d:/cc/arm-yagarto-5.4.2016q3/bin/../lib/gcc/arm-none-eabi/5.4.1/armv7-m\libgcc.a(_arm_addsubdf3.o)
                                                  obj/uc_libc_dev/misc/utils.o
__aeabi_dcmpeq                                    d:/cc/arm-yagarto-5.4.2016q3/bin/../lib/gcc/arm-none-eabi/5.4.1/armv7-m\libgcc.a(_arm_cmpdf2.o)
                                                  obj/uc_libc_dev/stdio/stdio_uc.o
__aeabi_dcmpge                                    d:/cc/arm-yagarto-5.4.2016q3/bin/../lib/gcc/arm-none-eabi/5.4.1/armv7-m\libgcc.a(_arm_cmpdf2.o)
__aeabi_dcmpgt                                    d:/cc/arm-yagarto-5.4.2016q3/bin/../lib/gcc/arm-none-eabi/5.4.1/armv7-m\libgcc.a(_arm_cmpdf2.o)
                                                  obj/uc_libc_dev/stdio/stdio_uc.o
__aeabi_dcmple                                    d:/cc/arm-yagarto-5.4.2016q3/bin/../lib/gcc/arm-none-eabi/5.4.1/armv7-m\libgcc.a(_arm_cmpdf2.o)
__aeabi_dcmplt                                    d:/cc/arm-yagarto-5.4.2016q3/bin/../lib/gcc/arm-none-eabi/5.4.1/armv7-m\libgcc.a(_arm_cmpdf2.o)
                                                  obj/uc_libc_dev/stdio/stdio_uc.o
__aeabi_ddiv                                      d:/cc/arm-yagarto-5.4.2016q3/bin/../lib/gcc/arm-none-eabi/5.4.1/armv7-m\libgcc.a(_arm_muldivdf3.o)
                                                  obj/uc_libc_dev/stdio/stdio_uc.o
                                                  obj/uc_libc_dev/_arch/arm_lpc/uart/uart0_irq.o
__aeabi_dmul                                      d:/cc/arm-yagarto-5.4.2016q3/bin/../lib/gcc/arm-none-eabi/5.4.1/armv7-m\libgcc.a(_arm_muldivdf3.o)
                                                  obj/uc_libc_dev/misc/utils.o
                                                  obj/uc_libc_dev/stdio/stdio_uc.o
                                                  obj/uc_libc_dev/_arch/arm_lpc/uart/uart0_irq.o
__aeabi_drsub                                     d:/cc/arm-yagarto-5.4.2016q3/bin/../lib/gcc/arm-none-eabi/5.4.1/armv7-m\libgcc.a(_arm_addsubdf3.o)
__aeabi_dsub                                      d:/cc/arm-yagarto-5.4.2016q3/bin/../lib/gcc/arm-none-eabi/5.4.1/armv7-m\libgcc.a(_arm_addsubdf3.o)
                                                  obj/uc_libc_dev/stdio/stdio_uc.o
__aeabi_f2d                                       d:/cc/arm-yagarto-5.4.2016q3/bin/../lib/gcc/arm-none-eabi/5.4.1/armv7-m\libgcc.a(_arm_addsubdf3.o)
                                                  obj/uc_libc_dev/_arch/arm_lpc/uart/uart0_irq.o
__aeabi_fadd                                      d:/cc/arm-yagarto-5.4.2016q3/bin/../lib/gcc/arm-none-eabi/5.4.1/armv7-m\libgcc.a(_arm_addsubsf3.o)
                                                  obj/uc_libc_dev/_arch/arm_lpc/uart/uart0_irq.o
__aeabi_fdiv                                      d:/cc/arm-yagarto-5.4.2016q3/bin/../lib/gcc/arm-none-eabi/5.4.1/armv7-m\libgcc.a(_arm_muldivsf3.o)
                                                  obj/uc_libc_dev/_arch/arm_lpc/uart/uart0_irq.o
__aeabi_fmul                                      d:/cc/arm-yagarto-5.4.2016q3/bin/../lib/gcc/arm-none-eabi/5.4.1/armv7-m\libgcc.a(_arm_muldivsf3.o)
                                                  obj/uc_libc_dev/_arch/arm_lpc/uart/uart0_irq.o
__aeabi_frsub                                     d:/cc/arm-yagarto-5.4.2016q3/bin/../lib/gcc/arm-none-eabi/5.4.1/armv7-m\libgcc.a(_arm_addsubsf3.o)
__aeabi_fsub                                      d:/cc/arm-yagarto-5.4.2016q3/bin/../lib/gcc/arm-none-eabi/5.4.1/armv7-m\libgcc.a(_arm_addsubsf3.o)
__aeabi_i2d                                       d:/cc/arm-yagarto-5.4.2016q3/bin/../lib/gcc/arm-none-eabi/5.4.1/armv7-m\libgcc.a(_arm_addsubdf3.o)
                                                  obj/uc_libc_dev/misc/utils.o
                                                  obj/uc_libc_dev/stdio/stdio_uc.o
                                                  obj/uc_libc_dev/_arch/arm_lpc/uart/uart0_irq.o
__aeabi_i2f                                       d:/cc/arm-yagarto-5.4.2016q3/bin/../lib/gcc/arm-none-eabi/5.4.1/armv7-m\libgcc.a(_arm_addsubsf3.o)
                                                  obj/uc_libc_dev/_arch/arm_lpc/uart/uart0_irq.o
__aeabi_l2d                                       d:/cc/arm-yagarto-5.4.2016q3/bin/../lib/gcc/arm-none-eabi/5.4.1/armv7-m\libgcc.a(_arm_addsubdf3.o)
__aeabi_l2f                                       d:/cc/arm-yagarto-5.4.2016q3/bin/../lib/gcc/arm-none-eabi/5.4.1/armv7-m\libgcc.a(_arm_addsubsf3.o)
__aeabi_ui2d                                      d:/cc/arm-yagarto-5.4.2016q3/bin/../lib/gcc/arm-none-eabi/5.4.1/armv7-m\libgcc.a(_arm_addsubdf3.o)
__aeabi_ui2f                                      d:/cc/arm-yagarto-5.4.2016q3/bin/../lib/gcc/arm-none-eabi/5.4.1/armv7-m\libgcc.a(_arm_addsubsf3.o)
__aeabi_ul2d                                      d:/cc/arm-yagarto-5.4.2016q3/bin/../lib/gcc/arm-none-eabi/5.4.1/armv7-m\libgcc.a(_arm_addsubdf3.o)
__aeabi_ul2f                                      d:/cc/arm-yagarto-5.4.2016q3/bin/../lib/gcc/arm-none-eabi/5.4.1/armv7-m\libgcc.a(_arm_addsubsf3.o)
__ascii_mbtowc                                    d:/cc/arm-yagarto-5.4.2016q3/bin/../lib/gcc/arm-none-eabi/5.4.1/../../../../arm-none-eabi/lib/armv7-m\libc.a(lib_a-mbtowc_r.o)
                                                  d:/cc/arm-yagarto-5.4.2016q3/bin/../lib/gcc/arm-none-eabi/5.4.1/../../../../arm-none-eabi/lib/armv7-m\libc.a(lib_a-locale.o)
__ascii_wctomb                                    d:/cc/arm-yagarto-5.4.2016q3/bin/../lib/gcc/arm-none-eabi/5.4.1/../../../../arm-none-eabi/lib/armv7-m\libc.a(lib_a-wctomb_r.o)
                                                  d:/cc/arm-yagarto-5.4.2016q3/bin/../lib/gcc/arm-none-eabi/5.4.1/../../../../arm-none-eabi/lib/armv7-m\libc.a(lib_a-locale.o)
__cmpdf2                                          d:/cc/arm-yagarto-5.4.2016q3/bin/../lib/gcc/arm-none-eabi/5.4.1/armv7-m\libgcc.a(_arm_cmpdf2.o)
__divdf3                                          d:/cc/arm-yagarto-5.4.2016q3/bin/../lib/gcc/arm-none-eabi/5.4.1/armv7-m\libgcc.a(_arm_muldivdf3.o)
__divsf3                                          d:/cc/arm-yagarto-5.4.2016q3/bin/../lib/gcc/arm-none-eabi/5.4.1/armv7-m\libgcc.a(_arm_muldivsf3.o)
__eqdf2                                           d:/cc/arm-yagarto-5.4.2016q3/bin/../lib/gcc/arm-none-eabi/5.4.1/armv7-m\libgcc.a(_arm_cmpdf2.o)
__extendsfdf2                                     d:/cc/arm-yagarto-5.4.2016q3/bin/../lib/gcc/arm-none-eabi/5.4.1/armv7-m\libgcc.a(_arm_addsubdf3.o)
__fixdfsi                                         d:/cc/arm-yagarto-5.4.2016q3/bin/../lib/gcc/arm-none-eabi/5.4.1/armv7-m\libgcc.a(_arm_fixdfsi.o)
__floatdidf                                       d:/cc/arm-yagarto-5.4.2016q3/bin/../lib/gcc/arm-none-eabi/5.4.1/armv7-m\libgcc.a(_arm_addsubdf3.o)
__floatdisf                                       d:/cc/arm-yagarto-5.4.2016q3/bin/../lib/gcc/arm-none-eabi/5.4.1/armv7-m\libgcc.a(_arm_addsubsf3.o)
__floatsidf                                       d:/cc/arm-yagarto-5.4.2016q3/bin/../lib/gcc/arm-none-eabi/5.4.1/armv7-m\libgcc.a(_arm_addsubdf3.o)
__floatsisf                                       d:/cc/arm-yagarto-5.4.2016q3/bin/../lib/gcc/arm-none-eabi/5.4.1/armv7-m\libgcc.a(_arm_addsubsf3.o)
__floatundidf                                     d:/cc/arm-yagarto-5.4.2016q3/bin/../lib/gcc/arm-none-eabi/5.4.1/armv7-m\libgcc.a(_arm_addsubdf3.o)
__floatundisf                                     d:/cc/arm-yagarto-5.4.2016q3/bin/../lib/gcc/arm-none-eabi/5.4.1/armv7-m\libgcc.a(_arm_addsubsf3.o)
__floatunsidf                                     d:/cc/arm-yagarto-5.4.2016q3/bin/../lib/gcc/arm-none-eabi/5.4.1/armv7-m\libgcc.a(_arm_addsubdf3.o)
__floatunsisf                                     d:/cc/arm-yagarto-5.4.2016q3/bin/../lib/gcc/arm-none-eabi/5.4.1/armv7-m\libgcc.a(_arm_addsubsf3.o)
__gedf2                                           d:/cc/arm-yagarto-5.4.2016q3/bin/../lib/gcc/arm-none-eabi/5.4.1/armv7-m\libgcc.a(_arm_cmpdf2.o)
__global_locale                                   d:/cc/arm-yagarto-5.4.2016q3/bin/../lib/gcc/arm-none-eabi/5.4.1/../../../../arm-none-eabi/lib/armv7-m\libc.a(lib_a-locale.o)
                                                  d:/cc/arm-yagarto-5.4.2016q3/bin/../lib/gcc/arm-none-eabi/5.4.1/../../../../arm-none-eabi/lib/armv7-m\libc.a(lib_a-wctomb_r.o)
                                                  d:/cc/arm-yagarto-5.4.2016q3/bin/../lib/gcc/arm-none-eabi/5.4.1/../../../../arm-none-eabi/lib/armv7-m\libc.a(lib_a-mbtowc_r.o)
__gtdf2                                           d:/cc/arm-yagarto-5.4.2016q3/bin/../lib/gcc/arm-none-eabi/5.4.1/armv7-m\libgcc.a(_arm_cmpdf2.o)
__ledf2                                           d:/cc/arm-yagarto-5.4.2016q3/bin/../lib/gcc/arm-none-eabi/5.4.1/armv7-m\libgcc.a(_arm_cmpdf2.o)
__locale_ctype_ptr                                d:/cc/arm-yagarto-5.4.2016q3/bin/../lib/gcc/arm-none-eabi/5.4.1/../../../../arm-none-eabi/lib/armv7-m\libc.a(lib_a-locale.o)
                                                  obj/uc_libc_dev/cli/cli.o
                                                  obj/uc_libc_dev/misc/utils.o
__locale_ctype_ptr_l                              d:/cc/arm-yagarto-5.4.2016q3/bin/../lib/gcc/arm-none-eabi/5.4.1/../../../../arm-none-eabi/lib/armv7-m\libc.a(lib_a-locale.o)
__locale_mb_cur_max                               d:/cc/arm-yagarto-5.4.2016q3/bin/../lib/gcc/arm-none-eabi/5.4.1/../../../../arm-none-eabi/lib/armv7-m\libc.a(lib_a-locale.o)
__ltdf2                                           d:/cc/arm-yagarto-5.4.2016q3/bin/../lib/gcc/arm-none-eabi/5.4.1/armv7-m\libgcc.a(_arm_cmpdf2.o)
__muldf3                                          d:/cc/arm-yagarto-5.4.2016q3/bin/../lib/gcc/arm-none-eabi/5.4.1/armv7-m\libgcc.a(_arm_muldivdf3.o)
__mulsf3                                          d:/cc/arm-yagarto-5.4.2016q3/bin/../lib/gcc/arm-none-eabi/5.4.1/armv7-m\libgcc.a(_arm_muldivsf3.o)
__nedf2                                           d:/cc/arm-yagarto-5.4.2016q3/bin/../lib/gcc/arm-none-eabi/5.4.1/armv7-m\libgcc.a(_arm_cmpdf2.o)
__subdf3                                          d:/cc/arm-yagarto-5.4.2016q3/bin/../lib/gcc/arm-none-eabi/5.4.1/armv7-m\libgcc.a(_arm_addsubdf3.o)
__subsf3                                          d:/cc/arm-yagarto-5.4.2016q3/bin/../lib/gcc/arm-none-eabi/5.4.1/armv7-m\libgcc.a(_arm_addsubsf3.o)
_bss                                              obj/uc_libc_dev/_arch/arm_lpc/common/startup/startup.o
_cols                                             obj/uc_libc_dev/display/liquid_crystal.o
_ctype_                                           d:/cc/arm-yagarto-5.4.2016q3/bin/../lib/gcc/arm-none-eabi/5.4.1/../../../../arm-none-eabi/lib/armv7-m\libc.a(lib_a-ctype_.o)
                                                  d:/cc/arm-yagarto-5.4.2016q3/bin/../lib/gcc/arm-none-eabi/5.4.1/../../../../arm-none-eabi/lib/armv7-m\libc.a(lib_a-locale.o)
_data                                             obj/uc_libc_dev/_arch/arm_lpc/common/startup/startup.o
_displaycontrol                                   obj/uc_libc_dev/display/liquid_crystal.o
_displayfunction                                  obj/uc_libc_dev/display/liquid_crystal.o
_displaymode                                      obj/uc_libc_dev/display/liquid_crystal.o
_ebss                                             obj/uc_libc_dev/_arch/arm_lpc/common/startup/startup.o
_edata                                            obj/uc_libc_dev/_arch/arm_lpc/common/startup/startup.o
_etext                                            obj/uc_libc_dev/_arch/arm_lpc/common/startup/startup.o
_exit                                             obj/uc_libc_dev/_arch/arm_lpc/common/arm.o
_global_impure_ptr                                d:/cc/arm-yagarto-5.4.2016q3/bin/../lib/gcc/arm-none-eabi/5.4.1/../../../../arm-none-eabi/lib/armv7-m\libc.a(lib_a-impure.o)
_impure_ptr                                       d:/cc/arm-yagarto-5.4.2016q3/bin/../lib/gcc/arm-none-eabi/5.4.1/../../../../arm-none-eabi/lib/armv7-m\libc.a(lib_a-impure.o)
                                                  d:/cc/arm-yagarto-5.4.2016q3/bin/../lib/gcc/arm-none-eabi/5.4.1/../../../../arm-none-eabi/lib/armv7-m\libc.a(lib_a-wctomb_r.o)
                                                  d:/cc/arm-yagarto-5.4.2016q3/bin/../lib/gcc/arm-none-eabi/5.4.1/../../../../arm-none-eabi/lib/armv7-m\libc.a(lib_a-mbtowc_r.o)
                                                  d:/cc/arm-yagarto-5.4.2016q3/bin/../lib/gcc/arm-none-eabi/5.4.1/../../../../arm-none-eabi/lib/armv7-m\libc.a(lib_a-locale.o)
_mbtowc_r                                         d:/cc/arm-yagarto-5.4.2016q3/bin/../lib/gcc/arm-none-eabi/5.4.1/../../../../arm-none-eabi/lib/armv7-m\libc.a(lib_a-mbtowc_r.o)
_numlines                                         obj/uc_libc_dev/display/liquid_crystal.o
_row_offsets                                      obj/uc_libc_dev/display/liquid_crystal.o
_setlocale_r                                      d:/cc/arm-yagarto-5.4.2016q3/bin/../lib/gcc/arm-none-eabi/5.4.1/../../../../arm-none-eabi/lib/armv7-m\libc.a(lib_a-locale.o)
_stack                                            obj/uc_libc_dev/_arch/arm_lpc/common/vic_cortexm3.o
_start                                            obj/uc_libc_dev/_arch/arm_lpc/common/startup/startup.o
                                                  obj/uc_libc_dev/_arch/arm_lpc/common/vic_cortexm3.o
_wctomb_r                                         d:/cc/arm-yagarto-5.4.2016q3/bin/../lib/gcc/arm-none-eabi/5.4.1/../../../../arm-none-eabi/lib/armv7-m\libc.a(lib_a-wctomb_r.o)
adc_ISR                                           obj/uc_libc_dev/_arch/arm_lpc/common/vic_cortexm3.o
app_Init                                          obj/app.o
                                                  obj/main.o
app_Process                                       obj/app.o
                                                  obj/main.o
app_Tick                                          obj/app.o
                                                  obj/main.o
arm_Init                                          obj/uc_libc_dev/_arch/arm_lpc/common/arm.o
                                                  obj/uc_libc_dev/_arch/arm_lpc/common/startup/startup.o
armsDown                                          obj/app.o
armsUp                                            obj/app.o
beep_Init                                         obj/uc_libc_dev/sound/beep/beep.o
                                                  obj/main.o
beep_Play                                         obj/uc_libc_dev/sound/beep/beep.o
                                                  obj/prompt.o
                                                  obj/app.o
beep_Playing                                      obj/uc_libc_dev/sound/beep/beep.o
beep_Stop                                         obj/uc_libc_dev/sound/beep/beep.o
beep_Tick                                         obj/uc_libc_dev/sound/beep/beep.o
                                                  obj/app.o
bod_ISR                                           obj/uc_libc_dev/_arch/arm_lpc/common/vic_cortexm3.o
buffer_AddToEnd                                   obj/uc_libc_dev/misc/buffer.o
                                                  obj/uc_libc_dev/_arch/arm_lpc/uart/uart0_irq.o
buffer_Clear                                      obj/uc_libc_dev/misc/buffer.o
                                                  obj/uc_libc_dev/_arch/arm_lpc/uart/uart0_irq.o
buffer_DumpFromFront                              obj/uc_libc_dev/misc/buffer.o
buffer_GetAtIndex                                 obj/uc_libc_dev/misc/buffer.o
buffer_GetFromFront                               obj/uc_libc_dev/misc/buffer.o
                                                  obj/uc_libc_dev/_arch/arm_lpc/uart/uart0_irq.o
buffer_Init                                       obj/uc_libc_dev/misc/buffer.o
                                                  obj/uc_libc_dev/_arch/arm_lpc/uart/uart0_irq.o
buffer_IsEmpty                                    obj/uc_libc_dev/misc/buffer.o
                                                  obj/uc_libc_dev/_arch/arm_lpc/uart/uart0_irq.o
buffer_IsNotFull                                  obj/uc_libc_dev/misc/buffer.o
buffer_dump                                       obj/uc_libc_dev/misc/utils.o
busFault_ISR                                      obj/uc_libc_dev/_arch/arm_lpc/common/vic_cortexm3.o
canAct_ISR                                        obj/uc_libc_dev/_arch/arm_lpc/common/vic_cortexm3.o
can_ISR                                           obj/uc_libc_dev/_arch/arm_lpc/common/vic_cortexm3.o
cli_ArgsDispatch                                  obj/uc_libc_dev/cli/cli.o
                                                  obj/prompt.o
cli_ArgsParse                                     obj/uc_libc_dev/cli/cli.o
                                                  obj/prompt.o
cli_GetLine                                       obj/uc_libc_dev/cli/cli.o
                                                  obj/prompt.o
cli_Help                                          obj/uc_libc_dev/cli/cli.o
                                                  obj/prompt.o
cmd_list_active                                   obj/uc_libc_dev/cli/cli.o
control                                           obj/prompt.o
                                                  obj/app.o
                                                  obj/main.o
date2str                                          obj/uc_libc_dev/stdio/stdio_uc.o
debugMon_ISR                                      obj/uc_libc_dev/_arch/arm_lpc/common/vic_cortexm3.o
delay                                             obj/uc_libc_dev/_arch/arm_lpc/timer/delay.o
                                                  obj/uc_libc_dev/display/portable/arm_lpc/lcd_drv.o
                                                  obj/uc_libc_dev/display/liquid_crystal.o
                                                  obj/main.o
dma_ISR                                           obj/uc_libc_dev/_arch/arm_lpc/common/vic_cortexm3.o
doprint                                           obj/uc_libc_dev/stdio/stdio_uc.o
                                                  obj/uc_libc_dev/display/liquid_crystal.o
eeprom_ISR                                        obj/uc_libc_dev/_arch/arm_lpc/common/vic_cortexm3.o
eint0_ISR                                         obj/uc_libc_dev/_arch/arm_lpc/common/vic_cortexm3.o
eint1_ISR                                         obj/uc_libc_dev/_arch/arm_lpc/common/vic_cortexm3.o
eint2_ISR                                         obj/uc_libc_dev/_arch/arm_lpc/common/vic_cortexm3.o
eint3_ISR                                         obj/uc_libc_dev/_arch/arm_lpc/common/vic_cortexm3.o
enet_ISR                                          obj/uc_libc_dev/_arch/arm_lpc/common/vic_cortexm3.o
frownie                                           obj/app.o
gKey_Init                                         obj/uc_libc_dev/keyboard/gkey.o
                                                  obj/main.o
gKey_Process                                      obj/uc_libc_dev/keyboard/gkey.o
                                                  obj/main.o
gKey_Tick                                         obj/uc_libc_dev/keyboard/gkey.o
                                                  obj/app.o
gVectors                                          obj/uc_libc_dev/_arch/arm_lpc/common/vic_cortexm3.o
gkey_FastInc                                      obj/uc_libc_dev/keyboard/gkey.o
                                                  obj/app.o
gpio_ISR                                          obj/uc_libc_dev/_arch/arm_lpc/common/vic_cortexm3.o
hardFault_ISR                                     obj/uc_libc_dev/_arch/arm_lpc/common/vic_cortexm3.o
heart                                             obj/app.o
hoursToMinutes                                    obj/uc_libc_dev/misc/utils.o
i2c0_ISR                                          obj/uc_libc_dev/_arch/arm_lpc/common/vic_cortexm3.o
i2c1_ISR                                          obj/uc_libc_dev/_arch/arm_lpc/common/vic_cortexm3.o
i2c2_ISR                                          obj/uc_libc_dev/_arch/arm_lpc/common/vic_cortexm3.o
i2s_ISR                                           obj/uc_libc_dev/_arch/arm_lpc/common/vic_cortexm3.o
lcd_AutoScroll                                    obj/uc_libc_dev/display/liquid_crystal.o
lcd_Blink                                         obj/uc_libc_dev/display/liquid_crystal.o
lcd_Clear                                         obj/uc_libc_dev/display/liquid_crystal.o
lcd_CreateChar                                    obj/uc_libc_dev/display/liquid_crystal.o
                                                  obj/app.o
lcd_Cursor                                        obj/uc_libc_dev/display/liquid_crystal.o
lcd_Display                                       obj/uc_libc_dev/display/liquid_crystal.o
lcd_Home                                          obj/uc_libc_dev/display/liquid_crystal.o
lcd_ISR                                           obj/uc_libc_dev/_arch/arm_lpc/common/vic_cortexm3.o
lcd_Init                                          obj/uc_libc_dev/display/liquid_crystal.o
                                                  obj/main.o
lcd_LeftToRight                                   obj/uc_libc_dev/display/liquid_crystal.o
lcd_NoAutoScroll                                  obj/uc_libc_dev/display/liquid_crystal.o
lcd_NoBlink                                       obj/uc_libc_dev/display/liquid_crystal.o
lcd_NoCursor                                      obj/uc_libc_dev/display/liquid_crystal.o
lcd_NoDisplay                                     obj/uc_libc_dev/display/liquid_crystal.o
lcd_PutChar                                       obj/uc_libc_dev/display/liquid_crystal.o
                                                  obj/app.o
                                                  obj/main.o
lcd_RightToLeft                                   obj/uc_libc_dev/display/liquid_crystal.o
lcd_ScrollDisplayLeft                             obj/uc_libc_dev/display/liquid_crystal.o
lcd_ScrollDisplayRight                            obj/uc_libc_dev/display/liquid_crystal.o
lcd_SetCursor                                     obj/uc_libc_dev/display/liquid_crystal.o
                                                  obj/app.o
lcd_config_ports                                  obj/uc_libc_dev/display/portable/arm_lpc/lcd_drv.o
                                                  obj/uc_libc_dev/display/liquid_crystal.o
lcd_printf                                        obj/uc_libc_dev/display/liquid_crystal.o
                                                  obj/app.o
lcd_printfInit                                    obj/uc_libc_dev/display/liquid_crystal.o
                                                  obj/main.o
lcd_read                                          obj/uc_libc_dev/display/portable/arm_lpc/lcd_drv.o
                                                  obj/uc_libc_dev/display/liquid_crystal.o
lcd_write                                         obj/uc_libc_dev/display/portable/arm_lpc/lcd_drv.o
                                                  obj/uc_libc_dev/display/liquid_crystal.o
ldebug_RegisterDev                                obj/uc_libc_dev/stdio/stdio_uc.o
                                                  obj/main.o
ledError_Blink                                    obj/uc_libc_dev/misc/led_error.o
ledError_Init                                     obj/uc_libc_dev/misc/led_error.o
                                                  obj/main.o
ledError_Tick                                     obj/uc_libc_dev/misc/led_error.o
                                                  obj/app.o
lerr_RegisterDev                                  obj/uc_libc_dev/stdio/stdio_uc.o
lgetchar                                          obj/uc_libc_dev/stdio/stdio_uc.o
                                                  obj/uc_libc_dev/cli/cli.o
lgetchar_RegisterDev                              obj/uc_libc_dev/stdio/stdio_uc.o
                                                  obj/main.o
lputchar                                          obj/uc_libc_dev/stdio/stdio_uc.o
lputchar_RegisterDev                              obj/uc_libc_dev/stdio/stdio_uc.o
                                                  obj/main.o
main                                              obj/main.o
                                                  obj/uc_libc_dev/_arch/arm_lpc/common/startup/startup.o
mcpwm_ISR                                         obj/uc_libc_dev/_arch/arm_lpc/common/vic_cortexm3.o
memManage_ISR                                     obj/uc_libc_dev/_arch/arm_lpc/common/vic_cortexm3.o
memset                                            d:/cc/arm-yagarto-5.4.2016q3/bin/../lib/gcc/arm-none-eabi/5.4.1/../../../../arm-none-eabi/lib/armv7-m\libc.a(lib_a-memset.o)
                                                  obj/uc_libc_dev/cli/cli.o
minutesToHours                                    obj/uc_libc_dev/misc/utils.o
nmi_ISR                                           obj/uc_libc_dev/_arch/arm_lpc/common/vic_cortexm3.o
nvic_SetIntHandler                                obj/uc_libc_dev/_arch/arm_lpc/common/vic_cortexm3.o
                                                  obj/main.o
nvic_clearPendingIRQ                              obj/uc_libc_dev/_arch/arm_lpc/common/vic_cortexm3.o
                                                  obj/uc_libc_dev/_arch/arm_lpc/uart/uart0_irq.o
nvic_disableIRQ                                   obj/uc_libc_dev/_arch/arm_lpc/common/vic_cortexm3.o
nvic_enableIRQ                                    obj/uc_libc_dev/_arch/arm_lpc/common/vic_cortexm3.o
                                                  obj/uc_libc_dev/_arch/arm_lpc/uart/uart0_irq.o
nvic_getActiveIRQ                                 obj/uc_libc_dev/_arch/arm_lpc/common/vic_cortexm3.o
nvic_getPendingIRQ                                obj/uc_libc_dev/_arch/arm_lpc/common/vic_cortexm3.o
nvic_setPendingIRQ                                obj/uc_libc_dev/_arch/arm_lpc/common/vic_cortexm3.o
nvic_setPriority                                  obj/uc_libc_dev/_arch/arm_lpc/common/vic_cortexm3.o
                                                  obj/uc_libc_dev/_arch/arm_lpc/uart/uart0_irq.o
onKeyDown                                         obj/app.o
                                                  obj/main.o
onKeyPress                                        obj/app.o
                                                  obj/main.o
onKeyUp                                           obj/app.o
                                                  obj/main.o
pendSV_ISR                                        obj/uc_libc_dev/_arch/arm_lpc/common/vic_cortexm3.o
pll0_ISR                                          obj/uc_libc_dev/_arch/arm_lpc/common/vic_cortexm3.o
pll1_ISR                                          obj/uc_libc_dev/_arch/arm_lpc/common/vic_cortexm3.o
prompt_Process                                    obj/prompt.o
                                                  obj/main.o
put_dump                                          obj/uc_libc_dev/misc/utils.o
put_dump16                                        obj/uc_libc_dev/misc/utils.o
                                                  obj/prompt.o
pwm0_ISR                                          obj/uc_libc_dev/_arch/arm_lpc/common/vic_cortexm3.o
pwm_ISR                                           obj/uc_libc_dev/_arch/arm_lpc/common/vic_cortexm3.o
qei_ISR                                           obj/uc_libc_dev/_arch/arm_lpc/common/vic_cortexm3.o
relay_Init                                        obj/app.o
relay_Set                                         obj/app.o
                                                  obj/prompt.o
relay_Tick                                        obj/app.o
rit_ISR                                           obj/uc_libc_dev/_arch/arm_lpc/common/vic_cortexm3.o
rprintf                                           obj/uc_libc_dev/stdio/stdio_uc.o
                                                  obj/uc_libc_dev/display/liquid_crystal.o
                                                  obj/uc_libc_dev/cli/cli.o
                                                  obj/uc_libc_dev/misc/utils.o
                                                  obj/prompt.o
                                                  obj/app.o
                                                  obj/main.o
                                                  obj/uc_libc_dev/_arch/arm_lpc/common/vic_cortexm3.o
rprintf_RegisterDev                               obj/uc_libc_dev/stdio/stdio_uc.o
                                                  obj/uc_libc_dev/display/liquid_crystal.o
                                                  obj/main.o
rtc_ISR                                           obj/uc_libc_dev/_arch/arm_lpc/common/vic_cortexm3.o
sFormatArgs                                       obj/uc_libc_dev/stdio/stdio_uc.o
secondsToHours                                    obj/uc_libc_dev/misc/utils.o
setlocale                                         d:/cc/arm-yagarto-5.4.2016q3/bin/../lib/gcc/arm-none-eabi/5.4.1/../../../../arm-none-eabi/lib/armv7-m\libc.a(lib_a-locale.o)
sformat                                           obj/uc_libc_dev/stdio/stdio_uc.o
smiley                                            obj/app.o
spi_ISR                                           obj/uc_libc_dev/_arch/arm_lpc/common/vic_cortexm3.o
ssp0_ISR                                          obj/uc_libc_dev/_arch/arm_lpc/common/vic_cortexm3.o
ssp1_ISR                                          obj/uc_libc_dev/_arch/arm_lpc/common/vic_cortexm3.o
ssp2_ISR                                          obj/uc_libc_dev/_arch/arm_lpc/common/vic_cortexm3.o
strcmp                                            d:/cc/arm-yagarto-5.4.2016q3/bin/../lib/gcc/arm-none-eabi/5.4.1/../../../../arm-none-eabi/lib/armv7-m\libc.a(lib_a-strcmp.o)
                                                  d:/cc/arm-yagarto-5.4.2016q3/bin/../lib/gcc/arm-none-eabi/5.4.1/../../../../arm-none-eabi/lib/armv7-m\libc.a(lib_a-locale.o)
                                                  obj/uc_libc_dev/cli/cli.o
                                                  obj/prompt.o
strlen                                            d:/cc/arm-yagarto-5.4.2016q3/bin/../lib/gcc/arm-none-eabi/5.4.1/../../../../arm-none-eabi/lib/armv7-m\libc.a(lib_a-strlen-stub.o)
                                                  obj/uc_libc_dev/display/liquid_crystal.o
                                                  obj/uc_libc_dev/cli/cli.o
sun                                               obj/app.o
svc_ISR                                           obj/uc_libc_dev/_arch/arm_lpc/common/vic_cortexm3.o
sysTick_ISR                                       obj/uc_libc_dev/_arch/arm_lpc/timer/systick.o
                                                  obj/uc_libc_dev/_arch/arm_lpc/common/vic_cortexm3.o
systime_ClearIntHandler                           obj/uc_libc_dev/_arch/arm_lpc/timer/systick.o
systime_GetElapsedTick                            obj/uc_libc_dev/_arch/arm_lpc/timer/systick.o
systime_GetTick                                   obj/uc_libc_dev/_arch/arm_lpc/timer/systick.o
systime_Init                                      obj/uc_libc_dev/_arch/arm_lpc/timer/systick.o
                                                  obj/main.o
systime_Pause                                     obj/uc_libc_dev/_arch/arm_lpc/timer/systick.o
systime_SetIntHandler                             obj/uc_libc_dev/_arch/arm_lpc/timer/systick.o
                                                  obj/main.o
time2str                                          obj/uc_libc_dev/stdio/stdio_uc.o
timeout_Check                                     obj/uc_libc_dev/_arch/arm_lpc/timer/systick.o
timeout_Init                                      obj/uc_libc_dev/_arch/arm_lpc/timer/systick.o
timer0_ISR                                        obj/uc_libc_dev/_arch/arm_lpc/common/vic_cortexm3.o
timer1_ISR                                        obj/uc_libc_dev/_arch/arm_lpc/common/vic_cortexm3.o
timer2_ISR                                        obj/uc_libc_dev/_arch/arm_lpc/common/vic_cortexm3.o
timer3_ISR                                        obj/uc_libc_dev/_arch/arm_lpc/common/vic_cortexm3.o
uart0_BasicPutChar                                obj/uc_libc_dev/_arch/arm_lpc/uart/uart0_irq.o
                                                  obj/main.o
uart0_BufferQtdRx                                 obj/uc_libc_dev/_arch/arm_lpc/uart/uart0_irq.o
uart0_BufferRxIsEmpty                             obj/uc_libc_dev/_arch/arm_lpc/uart/uart0_irq.o
uart0_ClearBufferRx                               obj/uc_libc_dev/_arch/arm_lpc/uart/uart0_irq.o
uart0_CountRxOverflow                             obj/uc_libc_dev/_arch/arm_lpc/uart/uart0_irq.o
uart0_EmptyTx                                     obj/uc_libc_dev/_arch/arm_lpc/uart/uart0_irq.o
uart0_FlushTx                                     obj/uc_libc_dev/_arch/arm_lpc/uart/uart0_irq.o
uart0_GetBufferRx                                 obj/uc_libc_dev/_arch/arm_lpc/uart/uart0_irq.o
uart0_GetChar                                     obj/uc_libc_dev/_arch/arm_lpc/uart/uart0_irq.o
                                                  obj/main.o
uart0_ISR                                         obj/uc_libc_dev/_arch/arm_lpc/uart/uart0_irq.o
                                                  obj/uc_libc_dev/_arch/arm_lpc/common/vic_cortexm3.o
uart0_Init                                        obj/uc_libc_dev/_arch/arm_lpc/uart/uart0_irq.o
                                                  obj/main.o
uart0_PutChar                                     obj/uc_libc_dev/_arch/arm_lpc/uart/uart0_irq.o
                                                  obj/main.o
uart0_PutString                                   obj/uc_libc_dev/_arch/arm_lpc/uart/uart0_irq.o
uart0_SetBaudrate                                 obj/uc_libc_dev/_arch/arm_lpc/uart/uart0_irq.o
uart0_SpaceTx                                     obj/uc_libc_dev/_arch/arm_lpc/uart/uart0_irq.o
uart0_WriteTx                                     obj/uc_libc_dev/_arch/arm_lpc/uart/uart0_irq.o
uart1_ISR                                         obj/uc_libc_dev/_arch/arm_lpc/common/vic_cortexm3.o
uart2_ISR                                         obj/uc_libc_dev/_arch/arm_lpc/common/vic_cortexm3.o
uart3_ISR                                         obj/uc_libc_dev/_arch/arm_lpc/common/vic_cortexm3.o
uart4_ISR                                         obj/uc_libc_dev/_arch/arm_lpc/common/vic_cortexm3.o
usageFault_ISR                                    obj/uc_libc_dev/_arch/arm_lpc/common/vic_cortexm3.o
usbAct_ISR                                        obj/uc_libc_dev/_arch/arm_lpc/common/vic_cortexm3.o
usbHost_ISR                                       obj/uc_libc_dev/_arch/arm_lpc/common/vic_cortexm3.o
wdt_ISR                                           obj/uc_libc_dev/_arch/arm_lpc/common/vic_cortexm3.o
xatof                                             obj/uc_libc_dev/misc/utils.o
xatoi                                             obj/uc_libc_dev/misc/utils.o
                                                  obj/prompt.o
